:100000002BC3000048C3000046C3000044C30000E7
:1000100042C3000040C300003EC300003CC30000D8
:100020003AC3000038C3000036C3000034C30000E8
:100030000C94983E30C300002EC300002CC3000077
:100040002AC3000028C300000C94843E24C300008F
:1000500022C3000020C300001EC300001CC3000018
:100060001AC3000018C3000016C3000014C3000028
:1000700012C3000010C300000EC300000CC3000038
:100080000AC3000008C3000006C30000510F980F08
:10009000C80FF80F50106B109B10D2103B110211BB
:1000A000760F7B0FCD10F710FC10890F8E0F930F7A
:1000B00088139313951397139A139D13B713B913BA
:1000C000C613D213D516DA16E816ED16F216F71681
:1000D000FC160117831B861B891B8C1B8F1B921B15
:1000E000951B981B432568257C258F259225A325E4
:1000F000B425D22559255C25C525C825CB255F25E6
:1001000062256525CF2AD42AD92ADE2AE32AE82ABD
:10011000ED2AF22AF72AFA2AAE2C192D3D2EA62E08
:10012000C52FF130D731CC32FB334A34AD34F734FC
:10013000FE345235A735AA35AD35B035B335B635B1
:10014000B935BC3558386E3884389B38B138C73823
:10015000DD38F33847394A394D3950395339563932
:1001600059395C399639AB39C039D339E639F43964
:10017000073A1A3A2D3A423A573A6C3A8B3AA43A2D
:10018000000000000000000004040404000400005B
:100190000A0A0A00000000000A0A1F0A1F0A0A00D1
:1001A000040F140E051E040018190204081303009E
:1001B0000C12140814120D000C04080000000000BA
:1001C00002040808080402000804020202040800ED
:1001D0000004150E150400000004041F04040000B0
:1001E000000000000C0408000000001F00000000D8
:1001F00000000000000C0C000001020408100000C8
:100200000E11131519110E00040C040404040E0041
:100210000E11010204081F001F02040201110E004A
:1002200002060A121F0202001F101E0101110E0019
:100230000608101E11110E001F0102040808080014
:100240000E11110E11110E000E11110F01020C00F2
:100250000001020408100000000C0C000C0408004F
:10026000020408100804020000001F001F00000024
:1002700008040201020408000E1101020400040037
:100280000E11010D15150E000E1111111F11110087
:100290001E11111E11111E000E11101010110E0052
:1002A0001C12111111121C001F10101E10101F0023
:1002B0001F10101E101010000E11101711110E003B
:1002C0001111111F111111000E04040404040E0079
:1002D0000702020202120C0011121418141211006B
:1002E0001010101010101F00111B15151111110006
:1002F00011111915131111000E11111111110E0008
:100300001E11111E101010000E11111115120D00EA
:100310001E11111E141211000F10100E01011E00EB
:100320001F040404040404001111111111110E0022
:1003300011111111110A04001111111115150E00DE
:1003400011110A040A1111001111110A0404040008
:100350001F01020408101F000E08080808080E00FC
:10036000110A1F041F0404000E02020202020E0002
:10037000040A1100000000000000000000001F003F
:10038000080400000000000000000E010F110F0023
:1003900010101E1111111E0000000E1010110E0081
:1003A00001010D1311110F0000000E111F100E009E
:1003B0000609081C08080800000F11110F010E00A3
:1003C000101016191111110004000C0404040E0081
:1003D0000200060202120C0010101214181412006F
:1003E0001808080808081C0000001A15151111004B
:1003F000000016191111110000000E1111110E004C
:1004000000001E111E10100000000F110F0101004E
:10041000000016191010100000000E100E011E0032
:1004200008081C08080906000000111111130D002E
:1004300000001111110A04000000111111150A0029
:100440000000110A040A1100000011110F010E0032
:1004500000001F0204081F00384444447C44440048
:100460007C404078444478007844447844447800A0
:100470007C404040404040000C14242424243C4450
:100480007C40407840407C005454543854545400CC
:10049000384404180444380044444C546444440030
:1004A00054444C5464444400444850605048440010
:1004B0001C24242424246400446C545444444400E4
:1004C0004444447C44444400384444444444380054
:1004D0007C444444444444007844447840404000D0
:1004E00038444040404438007C1010101010100078
:1004F0004444443C044438003854545438101000E8
:1005000044442810284444004444444444447E0263
:10051000444444443C0404005454545454547C0013
:100520005454545454547E026020203824243800FB
:100530004444446454546400404040784444780047
:100540003844041C0444380048545474545448003B
:100550003C44443C14244400000038043C443C0027
:1005600000007840784478000000784C784C78009F
:1005700000007840404040000000182828287C44B3
:10058000000038447C403C0000005454385454006F
:1005900000007804380478000000444C546444009F
:1005A0000010444C54644400000044487048440027
:1005B00000001C24444444000000446C5454440093
:1005C0000000484878484800000038444444380057
:1005D00000007848484848000000704870404000DB
:1005E000000038404040380000007C10101010001F
:1005F0000000484838087000000038545438100093
:1006000000004428102844000000484848487C0462
:1006100000004848380808000000545454547C0036
:100620000000545454547E02000060203C223C00E0
:1006300000004242724A7200000040407844780054
:10064000000070087808700000004C5272524C0094
:1006500000003C443C44440011241FBECFEFD0E1D5
:10066000DEBFCDBF16E0A0E0B1E0ECE3FEE800E0C5
:100670000BBF02C007900D92AE32B107D9F726E04A
:10068000AEE2B6E001C01D92AC3EB207E1F70E94B7
:10069000F63E0C941C47B4CCA89521E020937A0632
:1006A0002091D9063091DA062937310578F1209169
:1006B0009206309193062635310540F5BC012B5F3B
:1006C0003F4F30939306209392061092DA061092D1
:1006D000D90690912F06892F90E0880F991F80509E
:1006E00090400E94194780912F068F5F80932F06BC
:1006F000A49A80E185BBA8952FEF81EE94E021506C
:1007000080409040E1F700C0000015BA0895409184
:100710002E06E42FF0E0EE0FFF1FE050FF4F608148
:10072000718121E0240F20932E066817790720F5A8
:10073000E22FF0E0EE0FFF1FE050FF4F608171816C
:100740008617970760F455E0259F900111242250E9
:100750003109309393062093920640932E06209100
:10076000A3063091A4068217930730F484E190E049
:10077000909393068093920680918F0690E020914B
:100780009206309193068217930720F49093930674
:10079000809392060895CF93DF9300D000D0CDB719
:1007A000DEB78091630080FD6BC01C821B821A82C1
:1007B0001982BE016F5F7F4FCE0103960E943E42B9
:1007C0008B819C818531954098F08B819C8188320A
:1007D0009A4070F489819A818431954048F48091DF
:1007E000E0069091E10601969093E1068093E00681
:1007F0008B819C818937954098F08B819C818932CF
:100800009A4070F089819A818431954048F48091B2
:10081000E0069091E10601979093E1068093E0064F
:100820008B819C818531954098F08B819C818832A9
:100830009A4070F489819A81853C994048F0809172
:100840009206909193060196909393068093920658
:100850008B819C818937954098F08B819C8189326E
:100860009A4070F089819A81853C994048F0809146
:100870009206909193060197909393068093920627
:100880000F900F900F900F90DF91CF910895EF92FE
:10089000FF920F931F93CF93DF9300D000D0CDB77B
:1008A000DEB78091340190913501A0913601B0916D
:1008B000370189839A83AB83BC8303E02FEF3FEF3B
:1008C0004CED50E068E470E080E090E0EED72FEF70
:1008D0003FEF4CED50E06FE770E080E090E0E5D74F
:1008E0002FEF3FEF4CED50E066EB70E080E090E0E2
:1008F000DCD72FEF3FEF4CED50E06DEE70E080E085
:1009000090E0D3D72FEF3FEF45EA50E068E470E086
:1009100080E090E00E94CA0C2FEF3FEF45EA50E0E4
:1009200068E470E087E390E00E94CA0C2FEF3FEF8D
:1009300045EA50E068E470E08EE690E00E94CA0C60
:100940002FEF3FEF4EE650E068E470E085EA90E07C
:100950000E94CA0C2FEF3FEF48EA50E068E470E0D5
:100960008CED90E00E94CA0CEE24E394F12C2FE170
:1009700030E04FEF5FEF6AE570E08CE090E048D741
:1009800095E0E92EF12C2FE130E04FEF5FEF61E9C8
:1009900070E08CE090E03CD729E0E22EF12C2FE1D2
:1009A00030E04FEF5FEF68EC70E08CE090E030D724
:1009B00032E0E32EF12C2FE130E04FEF5FEF6AE5FC
:1009C00070E083E490E024D746E0E42EF12C2FE1A0
:1009D00030E04FEF5FEF61E970E083E490E018D71B
:1009E000E12CF12C2FE130E04FEF5FEF68EC70E08D
:1009F00083E490E00DD753E0E52EF12C2FE130E0B9
:100A00004FEF5FEF6AE570E08AE790E001D767E0BB
:100A1000E62EF12C2FE130E04FEF5FEF61E970E05F
:100A20008AE790E0F5D674E0E72EF12C2FE130E074
:100A30004FEF5FEF6AE570E081EB90E0E9D6E8E028
:100A4000EE2EF12C2FE130E04FEF5FEF61E970E027
:100A500081EB90E0DDD6E12CF12C2FE130E04FEF7F
:100A60005FEF68EC70E089E890E0D2D62FE130E0EB
:100A70004FEF5FEF68EC70E083EA90E0C9D6F3E0F7
:100A8000EF2E0FEF1FEF2CE330E04AE550E068E473
:100A900070E081EE90E0F3D7CE0101967C0102E098
:100AA0002FE130E040E058EF64E670E085EF90E041
:100AB00069D6A3E0EA2E0FEF1FEF20E530E04AE50C
:100AC00050E066E970E081EE90E0D9D700EE17E0E3
:100AD0002CED30E04EE051E06EEB70E085EF90E001
:100AE0000E94BC0D20EA30E04CE251E06CED70E079
:100AF0008EE091E00E94BC0D2CED30E04FE051E023
:100B00006EEB70E086EF90E00E94BC0D20EA30E0D2
:100B10004BE251E06CED70E08DE091E00E94BC0D85
:100B20002CED30E040E151E06EEB70E087EF90E0BB
:100B30000E94BC0D20EA30E04AE251E06CED70E02A
:100B40008CE091E00E94BC0D2CED30E041E151E0E1
:100B50006EEB70E088EF90E00E94BC0D20EA30E080
:100B60004AE251E06CED70E08BE091E00E94BC0D38
:100B7000B2E0EB2E0FEF1FEF2CE330E040EA50E045
:100B800063E070E080E590E07AD70F900F900F90CF
:100B90000F90DF91CF911F910F91FF90EF900895EB
:100BA000EF920F931F9383E0E82E0FEF1FEF22E3E6
:100BB00030E040EA50E064E670E084E190E05FD726
:100BC00020E530E04AE550E066E970E081EE90E033
:100BD00056D700EE17E02CED30E04EE051E06EEB22
:100BE00070E085EF90E0C8D720EA30E04CE251E0B9
:100BF0006CED70E08EE091E0BFD72CED30E04FE07F
:100C000051E06EEB70E086EF90E0B6D720EA30E07E
:100C10004BE251E06CED70E08DE091E0ADD72CED52
:100C200030E040E151E06EEB70E087EF90E0A4D758
:100C300020EA30E04AE251E06CED70E08CE091E0B7
:100C40009BD72CED30E041E151E06EEB70E088EF96
:100C500090E092D720EA30E04AE251E06CED70E09B
:100C60008BE091E089D71F910F91EF900895EF925B
:100C7000FF920F931F93CF93DF9300D000D0CDB797
:100C8000DEB77C018091630080FD22C11C821B8243
:100C90001A821982BE016F5F7F4FCE0103960E94B8
:100CA0003E420FE110E02DE230E042E550E06AE024
:100CB00070E08BE990E071D48B819C81893B9B40F3
:100CC00068F089819A81883D9E4040F489819A81AB
:100CD00089349D4018F089E0809325018B819C81A7
:100CE0008F32994090F08B819C81803F9A4068F4CC
:100CF00089819A81883D9E4040F489819A81893416
:100D00009D4018F085E0809325018B819C81853A78
:100D1000964090F08B819C818C3F984068F489814B
:100D20009A81883D9E4040F489819A8189349D4012
:100D300018F081E0809325018B819C81853A964053
:100D400090F08B819C818C3F984068F489819A81D6
:100D500088349D4040F489819A818D389A4018F0FA
:100D600082E0809325018B819C818F32994090F0A5
:100D70008B819C81803F9A4068F489819A81883474
:100D80009D4040F489819A818D389A4018F086E020
:100D9000809325018B819C81893B9B4060F08981F8
:100DA0009A8188349D4038F489819A818D389A409F
:100DB00010F0109225018B819C81893B9B4068F04B
:100DC00089819A818E3B9A4040F489819A818F3043
:100DD000964018F08AE0809325018B819C81853AAA
:100DE000964090F08B819C818C3F984068F489817B
:100DF0009A818C389A4040F489819A81813D97404C
:100E000018F083E0809325018B819C81853A964080
:100E100090F08B819C818C3F984068F489819A8105
:100E2000803D974040F489819A818D3D954018F02E
:100E300084E0809325018B819C818F32994090F0D2
:100E40008B819C81803F9A4068F489819A818C389B
:100E50009A4040F489819A81813D974018F087E05B
:100E6000809325018B819C818F32994090F08B81FA
:100E70009C81803F9A4068F489819A81803D9740A7
:100E800040F489819A818D3D954018F088E08093E7
:100E900025018B819C818D3D954068F08B819C81E3
:100EA0008C3F984040F489819A818C3D954018F49C
:100EB0008BE0809325018B819C818F32994040F09B
:100EC00089819A818C3D954018F48CE080932501AE
:100ED000809125018A3088F49091320691110DC0DD
:100EE0008093400690E0909331068093300682E034
:100EF000809332068EE080932501809125018A300F
:100F0000A9F48091400634E6839FC0011124909398
:100F100031068093300622E020933206E816F90667
:100F200010F08EE001C08BE08093250180912501B7
:100F30008A30C0F4909132069230A1F480933E063C
:100F40002091400690E04AE0249F800D911D1124DD
:100F5000909331068093300683E0809332068EE0D2
:100F600080932501209125012A3010F580913206C9
:100F70008330F1F420933F063091400680913E0685
:100F80004AE0849FC001112444E6349F800D911DE6
:100F90001124820F911D909331068093300621E039
:100FA00020933206E816F90668F48BE08093250159
:100FB000809125018B3049F4109231061092300651
:100FC000109232068EE080932501809125018C30AD
:100FD00019F483E2809325010F900F900F900F90EA
:100FE000DF91CF911F910F91FF90EF900895EF92B5
:100FF000FF920F93E0903006F09031062AE0E2165F
:10100000F10450F403E02FE130E04FEF5FEF66E1D1
:1010100070E088EC90E0FCD3E0903006F090310670
:10102000C7010B978935910550F403E02FE130E0BB
:101030004FEF5FEF66E170E084EB90E0E9D3E09082
:101040003006F0903106C7018456910984389340E8
:1010500050F403E02FE130E04FEF5FEF66E170E026
:101060008BE990E0D5D30F91FF90EF9008950F9307
:101070001F93CF93DF93EC018B01809125018E317B
:1010800018F48FE190E0FED3109331060093300600
:10109000809125018E3128F4FADBCE01E8DDA7DF4F
:1010A000F7CF8FE190E0EED380913006909131063A
:1010B000DF91CF911F910F9108958EE080932501CC
:1010C0000895EF92FF920F931F93CF93DF93CDB7C5
:1010D000DEB728970FB6F894DEBF0FBECDBF809164
:1010E000630080FD50C018861F821E821D82BE01D3
:1010F0006B5F7F4FCE0107960E943E420FE110E0EA
:101100002EE230E044E650E062E370E082E390E0FB
:1011100044D28F819885853A964090F08F8198854A
:101120008C389A4068F48D819E8184379E4040F4CB
:101130008D819E81813F9A4018F081E08093250146
:101140008F819885853A964088F08F8198858C3874
:101150009A4060F48D819E818C389A4038F48D815C
:101160009E818939984010F0109225018F819885D1
:101170008F32994040F08D819E818C3D954018F4CE
:101180008CE08093250180912501813011F48093BA
:10119000240180912401813061F580913801909182
:1011A0003901A0913A0189839A83AB83CE010196DC
:1011B0007C0104E02FE130E040EE57E062E370E0B4
:1011C00086E490E0DFD200EE17E02EE230E04DE45E
:1011D00050E067E670E087E190E0DFD10FE110E0DA
:1011E0002EE230E04DE450E067E670E086E690E005
:1011F000D4D180912501811102C0109224018091E7
:10120000240181112FC080913B0190913C01A0915C
:101210003D01B0913E0189839A83AB83BC8300E09A
:1012200018EF2EE230E04DE450E067E670E086E62D
:1012300090E0B3D10FE110E02EE230E04DE450E059
:1012400067E670E087E190E0A8D1CE0101967C01CD
:1012500004E02FE130E040E058EF62E370E087E324
:1012600090E090D2809125018C3019F483E2809334
:10127000250128960FB6F894DEBF0FBECDBFDF91D3
:10128000CF911F910F91FF90EF900895CF93C82FAA
:10129000809125018E3118F48FE190E0F3D2C09354
:1012A0002401809125018E3120F4A89579DC09DF95
:1012B000F8CF8FE190E0E6D280912401CF9108959C
:1012C000E2E6F0E090819E7F90839081946090832D
:1012D0009081977F9083A8988BBB8DE08A95F1F7DA
:1012E0000000A89A8081886080830895E2E6F0E09B
:1012F0009081916090839081946090839081977F9A
:101300009083A8988BBB8DE08A95F1F70000A89A8E
:101310008081886080830895CF93C82F892FE6DF6E
:101320008C2FCF91E3CFE2E6F0E020812160208393
:101330002081246020832081277F2083A8988BBB75
:1013400092BB8DE08A95F1F70000A89A80818860B1
:1013500080830895CF93C82F86E3B2DFC13049F070
:1013600030F0C23041F0C33059F488EE07C088E451
:1013700003C088E203C088E8B9DF04C0B7DF0BC050
:10138000CD7F49F48FEE90E090933606809335063A
:101390008FE391E008C08FE391E09093360680934D
:1013A00035068FEE90E09093340680933306CF910C
:1013B0000895CF93C82F8FEF8ABB81BB80936100C4
:1013C00081E084BBE2E6F0E080818260808381E09E
:1013D00077DF2FEF89E698E1215080409040E1F7D8
:1013E00000C0000080EC6CDF85E280DF81EC68DF0C
:1013F00081E17CDF85EC64DF8BE278DF8BE276DFF6
:1014000087EC5EDF86E872DF8C2FA4DF8AE358DF8B
:1014100085E06CDF81EB54DF80E068DF88E166DF28
:1014200086EB4EDF8AE062DF82E860DF87E25EDF24
:1014300081E146DF2FEF8DEE92E021508040904019
:10144000E1F700C0000089E2CF913ACF0F931F93DC
:10145000CF93DF938C01EB018AE232DFC8015CDFBE
:10146000CE01DF91CF911F910F9156CF0F931F9314
:10147000CF93DF938C01EB018BE222DFC8014CDFBD
:10148000CE01DF91CF911F910F9146CFCF93DF9384
:10149000EB01BC01DBDFBE01CE01E8DF8CE2DF91B6
:1014A000CF910ECFCF93DF93EA01F0DFCE01DF9132
:1014B000CF9139CF8F929F92AF92BF92CF92DF920E
:1014C000EF92FF920F931F93CF93DF93A895681726
:1014D000790738F48627972768277927862797275B
:1014E000A8952417350738F4422753272427352792
:1014F00042275327A895A0913506B0913606FC01E6
:10150000A817B90708F4FD016B01A617B70708F47F
:101510006D018091330690913406EA018417950796
:1015200008F4EC0179018217930708F47C01A8956F
:1015300096012F5F3F4F2E1B3F0BD7011196AC1B1F
:10154000BD0B0E94E4434B015C01B601CF017EDF7D
:10155000A895B701CE018ADF8CE2B2DEA895C12C36
:10156000D12C7601C814D904EA04FB0449F0C8015F
:10157000DADEA8958FEFC81AD80AE80AF80AF2CF7F
:10158000DF91CF911F910F91FF90EF90DF90CF905F
:10159000BF90AF909F908F9008950F931F93411528
:1015A000510579F02115310561F0FA01AB01615067
:1015B0007109260F371FBC01615071096E0F7F1F23
:1015C00079DF1F910F9108952F923F924F925F9272
:1015D0006F927F928F929F92AF92BF92CF92DF9243
:1015E000EF92FF920F931F93CF93DF93CDB7DEB7A8
:1015F00067970FB6F894DEBF0FBECDBF5C01798B45
:10160000688B598748873B872A870F83F12C28E00E
:10161000029FC00111241A821982E8E0F0E0FF8BDA
:10162000EE8B47019C01285F31093B8B2A8BFC0123
:10163000E052F340FD8BEC8BC888D98889819A8170
:10164000C80ED91E8A899B89EE89FF898E1B9F0B44
:101650009C0120583E4F3F872E878C899D898E1B89
:101660009F0BFC01E058FE4FFD87EC871E821D8218
:101670001C821B8287E0682E712C412C512C212C5E
:10168000312CFF81F7FD1EC0EE85FF85849190E02F
:10169000062C02C0959587950A94E2F780FF08C052
:1016A000088519859701A701B6018D819E8107C024
:1016B0000A851B859701A701B6018B819C818A0D44
:1016C0009B1D20C0FF81F03CF0F0EC85FD858491EE
:1016D00090E0062C02C0959587950A94E2F780FF6A
:1016E00009C0088519859701A701B601C501820DBA
:1016F000931D08C00A851B859701A701B601C50186
:10170000840D951D4ADF280C391C480C591CF1E04A
:101710006F1A71082B813C81280D391D3C832B8366
:101720008D819E81880D991D9E838D839FEF691603
:10173000790609F0A6CFEE89FF893197FF8BEE8BF2
:1017400029813A812E0D3F1D3A832983EF2B09F021
:1017500073CF67960FB6F894DEBF0FBECDBFDF9193
:10176000CF911F910F91FF90EF90DF90CF90BF909E
:10177000AF909F908F907F906F905F904F903F9031
:101780002F9008954F925F926F927F928F929F92C7
:10179000AF92BF92CF92DF92EF92FF920F931F937F
:1017A000CF93DF93EC016B014A013901102F88E0E0
:1017B000089F500111242701F20101912F010023FC
:1017C000B1F02091350630913606CE0108962817E3
:1017D000390720F4CA0CDB1CC1E0D0E0E12E9301F4
:1017E000A401B601CE01F0DECA0DDB1DE5CFDF910D
:1017F000CF911F910F91FF90EF90DF90CF90BF900E
:10180000AF909F908F907F906F905F904F900895D2
:101810006F927F928F929F92AF92BF92CF92DF9200
:10182000EF92FF920F93CF93DF9300D000D0CDB70C
:10183000DEB76C015B014A013901C70119821A82C6
:101840001B821C824AE0BE016F5F7F4F0E94F34300
:10185000CE0101967C019301A401B501C60192DF7E
:101860000F900F900F900F90DF91CF910F91FF90FD
:10187000EF90DF90CF90BF90AF909F908F907F9030
:101880006F9008950F931F93209133063091340683
:1018900060913506709136068C0140E050E080E0A2
:1018A00090E008DE1F910F9108956F927F928F92C2
:1018B0009F92AF92BF92CF92DF92EF92FF920F93DF
:1018C000CF93DF936C01EB017A0159014C01840E37
:1018D000951EB401BBDDBE01CE01C8DD8CE2F0DC9B
:1018E000612C712C6E147F0431F0C5011CDD8FEF6B
:1018F000681A780AF7CF023008F43EC0B401C60176
:10190000A5DDCE010196BC01B1DD8CE2D9DC612CF4
:10191000712C6E147F0431F0C50105DD8FEF681A5C
:10192000780AF7CF023041F1B401C6018FDDCE0154
:101930000296BC019BDD8CE2C3DC612C712C6E1421
:101940007F0431F0C501EFDC8FEF681A780AF7CF1A
:10195000033091F0B401C60179DDCE010396BC01DC
:1019600085DD8CE2ADDCC0E0D0E0CE15DF0521F0F6
:10197000C501D9DC2196F9CFDF91CF910F91FF906E
:10198000EF90DF90CF90BF90AF909F908F907F901F
:101990006F9008956F927F928F929F92AF92BF92B5
:1019A000CF92DF92EF92FF920F93CF93DF93EC01F0
:1019B0006B017A015901BC0149DD46018E0C9F1C67
:1019C000B401C60153DD8CE27BDC612C712C6E14FA
:1019D0007F0431F0C501A7DC8FEF681A780AF7CFD2
:1019E000023008F43EC0CE010196BC012FDDB401E7
:1019F000C6013CDD8CE264DC612C712C6E147F042A
:101A000031F0C50190DC8FEF681A780AF7CF023009
:101A100041F1CE010296BC0119DDB401C60126DDFB
:101A20008CE24EDC612C712C6E147F0431F0C50108
:101A30007ADC8FEF681A780AF7CF033091F0CE0185
:101A40000396BC0103DDB401C60110DD8CE238DC75
:101A5000C0E0D0E0CE15DF0521F0C50164DC2196A1
:101A6000F9CFDF91CF910F91FF90EF90DF90CF9062
:101A7000BF90AF909F908F907F906F9008956F92DE
:101A80007F928F929F92AF92BF92CF92DF92EF920E
:101A90000F931F93CF93DF936C015B01EA01390130
:101AA00048010E2D940101DFB301615071096A0DE7
:101AB0007B1D9401AE01C601F8DE9401A301B501BE
:101AC000C60168DFCE0101979401A301B5018C0D19
:101AD0009D1D60DFDF91CF911F910F91EF90DF90FF
:101AE000CF90BF90AF909F908F907F906F90089510
:101AF000EF92FF920F931F93CF93DF93EB018A0135
:101B00007901BC01640F751FA1DCBE01CE01AEDC02
:101B10008CE2D6DBC0E0D0E0C017D10721F0C701CE
:101B200002DC2196F9CFDF91CF911F910F91FF90A9
:101B3000EF900895EF92FF920F931F93CF93DF934F
:101B4000EB018A017901BC0181DCBE01600F711FCC
:101B5000CE018CDC8CE2B4DBC0E0D0E0C017D10752
:101B600021F0C701E0DB2196F9CFDF91CF911F91E2
:101B70000F91FF90EF9008952F923F924F925F92B6
:101B80006F927F928F929F92AF92BF92CF92DF928D
:101B9000EF92FF920F931F93CF93DF9300D000D06B
:101BA00000D0CDB7DEB76C017B015A0139012801A5
:101BB000261B370B3A8329838A01081B190B17FF51
:101BC00003C0119501951109CA14DB0420F02224E9
:101BD0002A94322C03C022242394312C89819A81A7
:101BE0009E838D8397FF05C09195819591099E8372
:101BF0008D832D813E813195219531093C832B8345
:101C0000E614F70428F08FEF9FEF9A83898304C0CE
:101C100021E030E03A83298348018D819E81881A32
:101C2000990AA201B701C6013DDCC401880F991FC2
:101C30002B813C818217930764F0CA14DB0499F06E
:101C40002D813E81821A930AC20CD31C08171907F2
:101C500044F3E614F70439F0800E911E89819A81CD
:101C6000E80EF91EDECF26960FB6F894DEBF0FBE43
:101C7000CDBFDF91CF911F910F91FF90EF90DF903B
:101C8000CF90BF90AF909F908F907F906F905F901C
:101C90004F903F902F900895AF92BF92CF92DF92D6
:101CA000EF92FF920F931F93CF93DF937C016B0111
:101CB000EA01590198011CDFB501615071096C0DF1
:101CC0007D1D9801AE01C70113DF9801A501B60182
:101CD000C70130DFCE0101979801A501B6018E0D35
:101CE0009F1DDF91CF911F910F91FF90EF90DF909B
:101CF000CF90BF90AF901ECF2F923F924F925F92A6
:101D00006F927F928F929F92AF92BF92CF92DF920B
:101D1000EF92FF920F931F93CF93DF931C012B0140
:101D2000690150E000271127041B150BC1E0D0E02A
:101D3000C41BD50BCC0FDD1FE12CF12CA6015701E4
:101D4000A40CB51CB5013101601A710AC301AADBEC
:101D5000A601B5014801820C931CC401A3DBA601B6
:101D60005201AE18BF08B501C4019CDBA601B50144
:101D7000C30198DBEC16FD06B4F08FEFE81AF80A01
:101D8000C701880F991F01968C0F9D1F22273327AB
:101D9000201B310BE216F30639F40C171D074CF02B
:101DA000C0E0D0E001C0CE010C171D0714F0EC011B
:101DB000C5CF0F5F1F4F9801220F331F2F5F3F4F7B
:101DC000820F931F1016110694F7DF91CF911F9188
:101DD0000F91FF90EF90DF90CF90BF90AF909F90CA
:101DE0008F907F906F905F904F903F902F900895CD
:101DF0004F925F926F927F928F929F92AF92BF921B
:101E0000CF92DF92EF92FF920F931F93CF93DF93C6
:101E1000EC015B014A01390128018601ADDE970121
:101E2000A201B301C401A8DE9501AE01B701C20150
:101E3000A3DEDF91CF911F910F91FF90EF90DF9084
:101E4000CF90BF90AF909F908F907F906F905F905A
:101E50004F900895CF93C82F8A3011F48DE0FADFA8
:101E60005D9BFECFCCB980E090E0CF910895CF92FA
:101E7000DF92EF92FF920F931F93CF93DF93CDB733
:101E8000DEB761970FB6F894DEBF0FBECDBF90E00E
:101E90008A30910508F0EFC1FC01EA5BFF4F0C941A
:101EA000DB43A8958AE0EFE3F1E0DE0111960190B3
:101EB0000D928A95E1F7CE0101967C0101E02FE1B8
:101EC00030E04FEF5FEF63E270E08AE090E05ADCD1
:101ED000A895E091D5068E2F90E08830910508F006
:101EE000CAC1FC01E05BFF4F0C94DB43B1EAEB2E6F
:101EF000B5E0FB2E04C0ACE9EA2EA5E0FA2E02E024
:101F00002FE130E04FEF5FEF6EE170E08BEE90E09D
:101F1000B1C1F4E7EF2EF5E0FF2E72C1EAE6EE2E36
:101F2000E5E0FE2E6DC170E6E72E75E0F72E68C184
:101F3000A89588E0E9E4F1E0DE01119601900D92A8
:101F40008A95E1F786E0E6EAF1E0DE011C96019071
:101F50000D928A95E1F7CE0101967C0101E02FE117
:101F600030E04FEF5FEF64E170E084E190E00ADC85
:101F7000CE010C967C012FE130E04FEF5FEF68E27D
:101F800070E08EE190E0FEDBA8958091830602C1AF
:101F9000A89587E0E1E5F1E0DE01119601900D9250
:101FA0008A95E1F786E0E6EAF1E0DE011C96019011
:101FB0000D928A95E1F7CE0101967C0101E02FE1B7
:101FC00030E04FEF5FEF64E170E084E190E0DADB56
:101FD000CE010C967C012FE130E04FEF5FEF68E21D
:101FE00070E08EE190E0CEDBA89580918A06D2C0A9
:101FF000A89587E0E8E5F1E0DE01119601900D92E9
:102000008A95E1F7CE0101967C0101E02FE130E0F5
:102010004FEF5FEF63E270E089E190E0B3DBA895FA
:102020002FE130E04FEF5FEF6EE170E08EEE90E079
:10203000A9DB40EEC42E47E0D42E51E6E52EF12C6C
:102040000EE110E021E630E04AE050E067E570E0A4
:1020500084E190E0CDDE06E311E021E630E042E2EB
:1020600051E067E570E08CE291E0C2DE60EAE62EC6
:10207000F12C0EE110E020EA30E04AE050E06AEA9C
:1020800070E084E190E0B4DE06E311E020EA30E0A5
:1020900042E251E06AEA70E08CE291E0A9DEEBC036
:1020A000A8958BE0EFE5F1E0DE01119601900D922D
:1020B0008A95E1F7CE0101967C0101E02FE130E045
:1020C0004FEF5FEF63E270E08FE090E05BDBA8959D
:1020D0008091DF065FC0A89586E0EAE6F1E0DE01C8
:1020E0001C9601900D928A95E1F78AE0E0E7F1E015
:1020F000DE01119601900D928A95E1F7CE010C96C2
:102100007C0101E02FE130E04FEF5FEF64E170E030
:1021100089E190E037DBCE0101967C012FE130E0D0
:102120004FEF5FEF63E270E08FE090E02BDBA8956C
:102130008091D4062FC0A89586E0EAE6F1E0DE01A2
:10214000119601900D928A95E1F785E0EAE7F1E0BA
:10215000DE011C9601900D928A95E1F7CE01019661
:102160007C0101E02FE130E04FEF5FEF64E170E0D0
:1021700089E190E007DBCE010C967C012FE130E095
:102180004FEF5FEF63E270E08FE190E0FBDAA8953C
:102190008091D106813059F110F532E9E32E35E016
:1021A000F32E2EC0A89588E0E3EEF1E0DE01119653
:1021B00001900D928A95E1F7CE0101967C0101E034
:1021C0002FE130E04FEF5FEF63E270E08FE090E0EF
:1021D000D9DAA89580919106813049F018F08230C3
:1021E00059F049C028E5E22E25E0F22E09C098E812
:1021F000E92E95E0F92E04C08EE7E82E85E0F82E52
:1022000001E030C0A8958BE0EFE7F1E0DE01119628
:1022100001900D928A95E1F785E0EAE8F1E0DE01B0
:102220001C9601900D928A95E1F7CE0101967C01F2
:1022300001E02FE130E04FEF5FEF64E170E08AE012
:1022400090E0A0DACE010C967C012FE130E04FEF58
:102250005FEF68E270E08EE190E094DAA895CE013D
:1022600001967C012FE130E04FEF5FEF6EE170E00F
:1022700086EE90E087DA61960FB6F894DEBF0FBE67
:10228000CDBFDF91CF911F910F91FF90EF90DF9025
:10229000CF900895CF93DF9300D000D0CDB7DEB7B5
:1022A0008091630080FD21C01C821B821A821982EA
:1022B000BE016F5F7F4FCE0103960E943E428B812D
:1022C0009C81853C994088F0A89589819A81843CBD
:1022D000994058F4A89589819A818D3D954028F0C0
:1022E000A89581E080937C06A8950F900F900F90A1
:1022F0000F90DF91CF910895CF93DF9300D000D05E
:10230000CDB7DEB7A8958091630080FD23C01C8205
:102310001B821A821982BE016F5F7F4FCE01039626
:102320000E943E428B819C81853C994098F0898136
:102330009A81843C994070F489819A818D3D9540C1
:1023400048F010927C068FE19EE40197F1F700C0FF
:102350000000A8950F900F900F900F90DF91CF91F4
:102360000895CF92DF92EF92FF920F931F93A8955B
:1023700080917C06811140C0A8950FE110E02CE40B
:1023800030E04EE650E06CE870E089E690E005D978
:1023900020E038EF48E264EB70E080EA90E0ACDCEB
:1023A00020E038EF47E264EB70E080EA90E0A4DCE4
:1023B00020E038EF4BE264EB70E080EA90E09CDCD8
:1023C00020E038EF45E264EB70E080EA90E094DCD6
:1023D00000E018EF23E230E045E050E065EA70E00D
:1023E00086E990E0DAD823E230E045E050E065EAA3
:1023F00070E085EA90E0D1D880917C06813009F0C8
:102400003EC0A8950FE110E02CE430E04EE650E02D
:102410006CE870E089E690E0C0D820EE37E048E252
:1024200064EB70E080EA90E067DC20EE37E047E2A2
:1024300064EB70E080EA90E05FDC20EE37E04BE296
:1024400064EB70E080EA90E057DC20EE37E045E294
:1024500064EB70E080EA90E04FDC80EEC82E87E00D
:10246000D82E94EBE92EF12C07EB10E028EC30E0AD
:1024700044E950E060EA70E084E990E0B9DC1F9143
:102480000F91FF90EF90DF90CF900895EF92FF9221
:102490000F931F93CF93DF93CDB7DEB764970FB63B
:1024A000F894DEBF0FBECDBFA8950FEF1FEF21E45C
:1024B00030E04FE550E065E070E085E090E0ECDB77
:1024C000A89521E430E04FE550E06BE470E085E052
:1024D00090E0E2DB2BE430E04FE550E061E970E0B2
:1024E00085E090E0D9DB89E0EFE8F1E0DE011196CC
:1024F00001900D928A95E1F785E0EAE8F1E0DE01CE
:10250000509601900D928A95E1F7CE0101967C01DB
:1025100001E02FE130E04FEF5FEF60E570E082E136
:1025200090E030D9CE0140967C012FE130E04FEFB2
:102530005FEF6AE570E083E290E024D90FEF1FEFD0
:1025400021E430E04FE550E065E070E08CED90E094
:10255000A3DB21E430E04FE550E06BE470E08CED6C
:1025600090E09ADB2BE430E04FE550E061E970E069
:102570008CED90E091DB86E0E8E9F1E0DE011A966F
:1025800001900D928A95E1F7CE0101967C0101E060
:102590002FE130E04FEF5FEF60E570E08BEE90E011
:1025A000F1D8CE010A967C012FE130E04FEF5FEFCA
:1025B0006AE570E08CEF90E0E5D88EE4E82E83E0E9
:1025C000F82E2FE130E04FEF5FEF66EE70E08AE02B
:1025D00090E0D8D8C6DE80917D0649DC64960FB6BF
:1025E000F894DEBF0FBECDBFDF91CF911F910F9149
:1025F000FF90EF900895EF92FF920F93CF93DF93A8
:10260000CDB7DEB7C458D1090FB6F894DEBF0FBE00
:10261000CDBF9AE0EFE3F1E0DE01AA59BF4F019090
:102620000D929A95E1F79EE0EEE9F1E0DE015E960B
:1026300001900D929A95E1F79EE0ECEAF1E0DE015F
:10264000509601900D929A95E1F79CE0EAEBF1E04B
:10265000DE01AB5BBF4F01900D929A95E1F79BE0D5
:10266000EFE5F1E0DE01AF5ABF4F01900D929A9570
:10267000E1F796E0EAE6F1E0DE01A158BF4F0190F4
:102680000D929A95E1F79AE0E0E7F1E0DE01A45AB5
:10269000BF4F01900D929A95E1F79DE0E6ECF1E0D5
:1026A000DE019C9601900D929A95E1F79FE0E3ED93
:1026B000F1E0DE01119601900D929A95E1F799E013
:1026C000E2EEF1E0DE01A059BF4F01900D929A9524
:1026D000E1F79CE0EBEEF1E0DE01D99601900D927E
:1026E0009A95E1F796E0E7EFF1E0DE01A758BF4FDA
:1026F00001900D929A95E1F7A89590E08A309105A6
:1027000008F06BC0FC01E85AFF4FCE010C94DB438C
:102710008A599F4F7C0102E02FE130E04FEF5FEFDD
:1027200062E870E030C04E9626C0409624C08B5BB5
:102730009F4F21C08F5A9F4F1EC081589F4F7C01D1
:1027400002E02FE130E04FEF5FEF6EE670E088E2ED
:1027500090E018D8CE01845A9F4F7C012FE130E0E1
:102760004FEF5FEF67E870E08FE090E034C08C9649
:1027700002C080599F4F7C0102E02FE130E04FEF13
:102780005FEF68E770E088E090E025C001967C018B
:1027900002E02FE130E04FEF5FEF68E770E082E0AA
:1027A00090E019C0C9967C0102E02FE130E04FEFC4
:1027B0005FEF6EE670E084E190E00E94C20BCE0114
:1027C00087589F4F7C012FE130E04FEF5FEF67E8C4
:1027D00070E08CE390E00E94C20BCC57DF4F0FB645
:1027E000F894DEBF0FBECDBFDF91CF910F91FF9068
:1027F000EF900895CF92DF92EF92FF920F931F9385
:10280000A89500EE17E021E430E048EC50E06AEAD9
:1028100070E085E090E00E94CD0A0FEF1FEF21E409
:1028200030E048EC50E063E270E085E090E034DABC
:102830008CE6E82E83E0F82E01E02FE130E040EE58
:1028400057E06CE370E088E290E00E94C20B0FEF6B
:102850001FEF20E530E040E550E065E070E08BEEF2
:1028600090E01ADA90EEC92E97E0D92E24E1E22EFC
:10287000F12C03E111E026E430E041E351E066E4AD
:1028800070E085EF90E0B4DA37E1E32EF12C24E438
:1028900030E04FE251E064E470E087EF90E0A8DAC6
:1028A0000FEF1FEF20E530E040E550E064E670E018
:1028B0008BEE90E0F1D945EAE42EF12C03E111E032
:1028C00023E730E041E351E063E770E085EF90E01B
:1028D0008FDA53EAE52EF12C25E730E04FE251E0A4
:1028E00065E770E087EF90E083DA60EBE62E65E065
:1028F000F62E02E020EE37E040E050E068EC70E0B9
:102900008DE290E00E94C20B1F910F91FF90EF901B
:10291000DF90CF900895CF92DF92EF92FF920F93C6
:102920001F93CF93DF93CDB7DEB765970FB6F894BB
:10293000DEBF0FBECDBFA8958FE0E3EDF1E0DE0175
:10294000119601900D928A95E1F786E0EDEFF1E0A6
:10295000DE01509601900D928A95E1F700EE17E0A6
:1029600021E430E048EC50E06AEA70E085E090E075
:102970000E94CD0A0FEF1FEF21E430E048EC50E059
:1029800063E270E085E090E087D9CE0101967C019A
:1029900001E02FE130E040EE57E06CE370E088E2C8
:1029A00090E00E94C20B0FEF1FEF20E530E040E502
:1029B00050E065E070E08BEE90E06ED980EEC82EBE
:1029C00087E0D82E94E1E92EF12C03E111E026E412
:1029D00030E041E351E066E470E085EF90E008DA32
:1029E00027E1E22EF12C24E430E04FE251E064E4F0
:1029F00070E087EF90E0FCD90FEF1FEF20E530E0AB
:102A000040E550E064E670E08BEE90E045D935EAB1
:102A1000E32EF12C03E111E023E730E041E351E044
:102A200063E770E085EF90E0E3D943EAE42EF12C10
:102A300025E730E04FE251E065E770E087EF90E096
:102A4000D7D9CE0140967C0102E020EE37E040E08D
:102A500050E068EC70E08DE290E00E94C20B659659
:102A60000FB6F894DEBF0FBECDBFDF91CF911F919F
:102A70000F91FF90EF90DF90CF900895CF92DF926B
:102A8000EF92FF920F931F93A89500EE17E021E4B9
:102A900030E048EC50E06AEA70E085E090E00E94A7
:102AA000CD0A0FEF1FEF21E430E048EC50E063E285
:102AB00070E085E090E0F0D887E4E82E85E0F82E1D
:102AC00001E02FE130E040EE57E06CE370E088E297
:102AD00090E00E94C20B0FEF1FEF20E530E040E5D1
:102AE00050E065E070E08BEE90E0D6D890EEC92E15
:102AF00097E0D92E24E1E22EF12C03E111E026E447
:102B000030E041E351E066E470E085EF90E070D999
:102B100037E1E32EF12C24E430E04FE251E064E4AD
:102B200070E087EF90E064D90FEF1FEF20E530E011
:102B300040E550E064E670E08BEE90E0ADD845EA09
:102B4000E42EF12C03E111E023E730E041E351E012
:102B500063E770E085EF90E04BD953EAE52EF12C66
:102B600025E730E04FE251E065E770E087EF90E065
:102B70003FD961ECE62E65E0F62E02E020EE37E06C
:102B800040E050E068EC70E08DE290E00E94C20B03
:102B90001F910F91FF90EF90DF90CF900895CF930A
:102BA000DF9300D000D0CDB7DEB78091630080FD09
:102BB00057C01C821B821A821982BE016F5F7F4F31
:102BC000CE0103960E943E428B819C8184319540C8
:102BD00068F489819A81843A964040F489819A8187
:102BE0008D32914018F082E080939F068B819C810A
:102BF0008937954090F08B819C81843C994068F4A2
:102C000089819A81843A964040F489819A818D32F3
:102C1000914018F083E080939F068B819C818932DC
:102C20009A4068F089819A8184379E4040F4898176
:102C30009A81813D974018F081E080939F068B81B7
:102C40009C81863F994060F48B819C8181349640C1
:102C500038F089819A81813D974010F010929F064B
:102C600080919F060F900F900F900F90DF91CF9162
:102C70000895CF92DF92EF92FF920F931F93CF931D
:102C8000DF9300D000D000D0CDB7DEB7A89586E0A6
:102C9000EDEFF1E0DE01119601900D928A95E1F7DA
:102CA00000EE17E021E430E048EC50E06AEA70E022
:102CB00085E090E00E94CD0A0FEF1FEF21E430E0A5
:102CC00048EC50E063E270E085E090E00E944C0E3A
:102CD00020E530E040E550E065E070E08BEE90E00C
:102CE0000E944C0EF0EECF2EF7E0DF2EA4E1EA2E8C
:102CF000F12C03E111E026E430E041E351E066E429
:102D000070E085EF90E074D8B7E1EB2EF12C24E46D
:102D100030E04FE251E064E470E087EF90E068D883
:102D20000FEF1FEF20E530E040E550E064E670E093
:102D30008BEE90E00E944C0E15EAE12EF12C03E19F
:102D400011E023E730E041E351E063E770E085EF15
:102D500090E04ED883EAE82EF12C25E730E04FE2F0
:102D600051E065E770E087EF90E042D8CE01019630
:102D70007C0102E020EE37E040E050E068EC70E0DB
:102D80008CE390E00E94C20B80917D06811148C0C7
:102D9000E091D5068E2F90E08830910508F040C074
:102DA000FC01EE59FF4F0C94DB43E1EAEE2EE5E027
:102DB000FE2E04C07CE9E72E75E0F72E02E02FE13D
:102DC00030E04FEF5FEF65E070E086E490E026C012
:102DD00062E9E62E65E0F62E18C058E8E52E55E0CB
:102DE000F52E13C04EE7E42E45E0F42E0EC034E776
:102DF000E32E35E0F32E09C02AE6E22E25E0F22E7E
:102E000004C090E6E92E95E0F92E02E02FE130E0D3
:102E10004FEF5FEF65E070E08EE190E00E94C20B43
:102E200080917D06813001F580918306813069F0C3
:102E300038F08230C9F41EE7E12E15E0F12E09C00A
:102E400082E9E82E85E0F82E04C008E8E02E05E0CF
:102E5000F02E02E02FE130E04FEF5FEF65E070E031
:102E60008EE190E00E94C20B80917D06823001F5D8
:102E700080918A06813069F038F08230C9F4FEE72B
:102E8000EF2EF5E0FF2E09C0B2E9EB2EB5E0FB2EE8
:102E900004C0A8E8EA2EA5E0FA2E02E02FE130E017
:102EA0004FEF5FEF65E070E08EE190E00E94C20BB3
:102EB00080917D06843001F58091DF06813069F0D4
:102EC00038F08230C9F46EE7E62E65E0F62E09C0D0
:102ED000E2E9EE2EE5E0FE2E04C078E8E72E75E08C
:102EE000F72E02E02FE130E04FEF5FEF65E070E09A
:102EF0008EE190E00E94C20B80917D06853001F545
:102F00008091D406813069F038F08230C9F43EE710
:102F1000E32E35E0F32E09C052E9E52E55E0F52EFB
:102F200004C048E8E42E45E0F42E02E02FE130E052
:102F30004FEF5FEF65E070E08EE190E00E94C20B22
:102F400080917D06863001F58091D106813069F04F
:102F500038F08230C9F48EE7E82E85E0F82E09C0FB
:102F600022E9E22E25E0F22E04C098E8E92E95E051
:102F7000F92E02E02FE130E04FEF5FEF65E070E007
:102F80008EE190E00E94C20B26960FB6F894DEBF49
:102F90000FBECDBFDF91CF911F910F91FF90EF90AA
:102FA000DF90CF900895EF92FF920F931F9380913F
:102FB0007506909176060A97A8F480914C068111C7
:102FC0000CC00FE110E02CE330E044E650E06BE48D
:102FD00070E08EE690E00E94CD0A81E080934C067E
:102FE00010927E0680917506909176060A978A3532
:102FF0009105A8F480917E0681110CC00FE110E0CC
:103000002CE330E044E650E06BE470E08EE690E0C4
:103010000E94CD0A81E080937E0610924C0680913A
:1030200075069091760684369105A0F080917E0613
:10303000813061F40FE110E02CE330E044E650E031
:103040006BE470E08EE690E00E94CD0A10927E065E
:1030500010924C0680917C06813079F4E0907506E0
:10306000F090760603E02FE130E04FEF5FEF64E68B
:1030700070E082E890E00E94080C80917C0681114B
:103080000FC0E0907506F090760603E02FE130E087
:1030900040E058EF64E670E082E890E00E94080C9F
:1030A0001F910F91FF90EF900895EF92FF920F9371
:1030B0001F938091A3069091A4060A97A8F480918B
:1030C0007406811111C00FE110E028E230E048E5FC
:1030D00050E06FEA70E088E090E00E94CD0A81E065
:1030E000809374061092D2068091A3069091A40654
:1030F00084369105D8F480917506909176060A97EA
:10310000A8F08091D206811111C00FE110E028E2F1
:1031100030E048E550E06FEA70E088E090E00E941F
:10312000CD0A81E08093D206109274068091A306A6
:103130009091A40684369105A0F08091D20681304A
:1031400061F40FE110E028E230E048E550E06FEA7A
:1031500070E088E090E00E94CD0A1092D2061092B2
:103160007406E090A306F090A40602E02FE130E0A0
:103170004FEF5FEF6EEB70E08EE190E00E94080C85
:103180001F910F91FF90EF900895EF92FF920F9390
:103190001F93809192068A30A8F480917B0681115A
:1031A0000CC00FE110E024E230E04AE550E064E6B4
:1031B00070E088E090E00E94CD0A81E080937B0679
:1031C00010928E06809192068A508A35A8F48091DA
:1031D0008E0681110CC00FE110E024E230E04AE5D8
:1031E00050E064E670E088E090E00E94CD0A81E063
:1031F00080938E0610927B06809192068436A1F40D
:1032000080918E06813061F40FE110E024E230E01D
:103210004AE550E064E670E088E090E00E94CD0A64
:1032200010927B0610928E0680919206843618F0DA
:1032300084E680939206E0909206F12C02E02FE162
:1032400030E04FEF5FEF6EE670E084E190E00E94C7
:10325000080C8091E0068A30A8F48091DB06811189
:1032600011C00FE110E024E230E04AE550E064E6EE
:1032700070E08FED90E00E94CD0A81E08093DB0644
:103280001092A5068091E0068A508A35A8F48091B4
:10329000A506811111C00FE110E024E230E04AE5FB
:1032A00050E064E670E08FED90E00E94CD0A81E08E
:1032B0008093A5061092DB068091E006843629F4FF
:1032C0001092DB061092A50602C0843618F084E640
:1032D0008093E006E090E006F12C02E02FE130E080
:1032E0004FEF5FEF6EE670E089EE90E00E94080C11
:1032F0001F910F91FF90EF9008957F928F929F9270
:10330000AF92BF92CF92DF92EF92FF920F931F93F3
:10331000CF93DF93EC016B015A014901702EA89500
:1033200080914F06909150060A97A8F48091D60696
:10333000811111C00FE110E02EE130E044E650E0D1
:1033400065507109CE0144970E94CD0A81E08093B7
:10335000D6061092980680914F06909150060A97D3
:103360008A359105C0F480919806811114C00FE14F
:1033700010E02EE130E044E650E0B60165507109FE
:10338000CE0144970E94CD0A81E080939806109266
:10339000D6061092770680914F069091500684369B
:1033A0009105C0F080917706811114C00FE110E003
:1033B0002EE130E044E650E0B60165507109CE01DF
:1033C00044970E94CD0A81E0809377061092980678
:1033D0001092D606E0904F06F0905006072D94010B
:1033E000A501B601CE010E94080CA895DF91CF91EE
:1033F0001F910F91FF90EF90DF90CF90BF90AF9013
:103400009F908F907F900895CF92DF92EF92FF92DE
:103410000F931F938FE190E00E94420CA89500EE5D
:1034200017E021E430E048EC50E06AEA70E085E023
:1034300090E00E94CD0A0FEF1FEF21E430E048EC4E
:1034400050E063E270E085E090E00E944C0E8EE375
:10345000E82E83E0F82E01E02FE130E040EE57E067
:103460006CE370E088E290E00E94C20B0FEF1FEF68
:1034700020E530E040E550E065E070E08BEE90E064
:103480000E944C0E90EEC92E97E0D92E24E1E22E38
:10349000F12C03E111E026E430E041E351E066E481
:1034A00070E085EF90E00E94F80E37E1E32EF12CFA
:1034B00024E430E04FE251E064E470E087EF90E014
:1034C0000E94F80E0FEF1FEF20E530E040E550E0DE
:1034D00064E670E08BEE90E00E944C0E45EAE42E2C
:1034E000F12C03E111E023E730E041E351E063E731
:1034F00070E085EF90E00E94F80E53EAE52EF12C83
:1035000025E730E04FE251E065E770E087EF90E0BB
:103510000E94F80E60EBE62E65E0F62E02E020EE4B
:1035200037E040E050E068EC70E08DE290E00E940F
:10353000C20B8FE19EE40197F1F700C000001F91DC
:103540000F91FF90EF90DF90CF900895A8958BEDAD
:1035500092E00E94F646813071F4A49A80E185BB26
:10356000A8952FEF82E597E0215080409040E1F749
:1035700000C0000015BAA8950895A8958BED92E0BB
:103580000E94F646813021F5A49A80E185BB2FEF99
:1035900032E597E0215030409040E1F700C0000054
:1035A000A89515BA2FEF32E597E0215030409040B2
:1035B000E1F700C00000A89585BB2FEF32E587E05A
:1035C000215030408040E1F700C00000A89515BAB6
:1035D0000895A8958BED92E00E94F646813009F09F
:1035E00048C0A49A80E185BBA8952FEF32E597E00B
:1035F000215030409040E1F700C00000A89515BA76
:10360000A8952FEF32E597E0215030409040E1F748
:1036100000C00000A89585BBA8952FEF32E597E084
:10362000215030409040E1F700C00000A89515BA45
:10363000A8952FEF32E597E0215030409040E1F718
:1036400000C00000A89585BB2FEF32E587E0215030
:1036500030408040E1F700C00000A89515BA9FEF08
:1036600022E537E0915020403040E1F700C00000F3
:10367000A89508951092E006BC9A8091E006880F04
:1036800081BF10929206139A80919206880F8093C0
:1036900086009FDF8DE490E09093D8068093D70654
:1036A0000895A895109293061092870610924A06E4
:1036B0001092A8061092840610927A061092940630
:1036C00010928D061092A20610924B06A8958CEDD2
:1036D00092E00E94FE469093890680938806A89502
:1036E00080917D0681112AC0A895E091D5068E2F84
:1036F00090E08830910510F5FC01E659FF4F4EE14E
:1037000050E00C94DB436CEB72E014C06EE972E0A5
:1037100011C060E872E00EC062E672E00BC064E4C3
:1037200072E008C066E272E005C068E072E002C0C4
:103730006AEE71E085E596E00E94E646A8958091E4
:103740007D068130D1F4A89580918306813069F09F
:1037500038F0823091F44EE150E060E971E009C048
:103760004EE150E06CEC71E004C04EE150E06EEAD6
:1037700071E085E596E00E94E646A89580917D0679
:103780008230D1F4A89580918A06813069F038F0B2
:10379000823091F44EE150E066E371E009C04EE101
:1037A00050E062E771E004C04EE150E064E571E092
:1037B00085E596E00E94E646A89580917D068430D6
:1037C000C9F48091DF06813069F038F0823091F4DD
:1037D0004EE150E06CED70E009C04EE150E068E170
:1037E00071E004C04EE150E06AEF70E085E596E0DC
:1037F0000E94E646A89580917D068530C9F48091A7
:10380000D406813069F038F0823091F44EE150E016
:1038100062E870E009C04EE150E06EEB70E004C079
:103820004EE150E060EA70E085E596E00E94E646F1
:10383000A89580917D068630C9F48091D1068130AB
:1038400069F038F0823091F44EE150E068E270E0C7
:1038500009C04EE150E064E670E004C04EE150E083
:1038600066E470E085E596E00E94E646A89587EC60
:1038700090E00197F1F700C000008091550690910B
:10388000560690934706809346068091570690917E
:1038900058069093970680939606809159068093D8
:1038A000DD0680915B068093820680915D068093A1
:1038B000AA0680915F0680938106809161068093BD
:1038C00090068091630680938F06809165068093B1
:1038D000420680916706909168069093CE06809389
:1038E000CD06809169068093A90680917D06873078
:1038F00021F480916B0680937D0680916D069091F6
:103900006E069093CC068093CB0680916F069091C3
:10391000700690935406809353068091710690919F
:1039200072069093790680937806A8950895809101
:10393000A806811117C0209181068091750690918B
:103940007606821B9109029768F482E38093E00671
:1039500081E08093A80680937A068091AA0681115F
:1039600001C0F4DD2091810630E06091DD064091D8
:10397000D9065091DA06649FC001659F900D11240D
:103980006AE070E00E94C743620F731F70934506A0
:10399000609344069091E006409146065091470698
:1039A0004617570720F450934506409344068091EC
:1039B0009006891710F48093E00680917506909127
:1039C00076062817390720F04817590728F155C0FF
:1039D0002091A2062111F8CF84179507A8F76091CE
:1039E0004406709145062091E0068617970750F42B
:1039F0002F5F253618F42093E006E6CF24E62093C7
:103A0000E00687C0222319F021502093E006209180
:103A1000E0062223C9F27DC02091E006222319F09E
:103A200021502093E006841B950B069768F0809147
:103A3000E0068A3010F41092E0068091E0068A30A9
:103A400018F08A508093E00680914B06811106C0E1
:103A500094DD81E080938D0680934B062091510682
:103A600030915206809188069091890682179307BB
:103A700020F400DE81E080937C0680918406811131
:103A80004FC04091CB065091CC068091810690E0CA
:103A90008417950708F044C0E0917506F09176060A
:103AA0004E175F0729F481E08093A2068093940665
:103AB0008091A2068130A1F560914D0670914E066D
:103AC00020915306309154066217730778F4809161
:103AD000E006E417F50728F48F5F853628F084E6C2
:103AE00003C0882319F081508093E006261737071A
:103AF000B8F41092A2068091D9069091DA06821B42
:103B0000930B9093DA068093D90681E08093840624
:103B100008954817590708F0B0CF2091E00680CFEC
:103B200008958091A806811117C08091810690E0C8
:103B300020917506309176068217930768F482E328
:103B40008093E00681E08093A80680937A068091B6
:103B5000AA06811101C0FADCE0918106F0E04091F3
:103B6000DD062091D9063091DA06429FC001439FBD
:103B7000900D11246AE070E00E94C7436E0F7F1F12
:103B800070934506609344069091E0064091460686
:103B9000509147064617570720F450934506409327
:103BA000440680919006891710F48093E0062091D6
:103BB000750630917606E217F307D0F48091A206DD
:103BC000811116C02417350798F46091440670914E
:103BD00045068091E0062617370728F48F5F853663
:103BE00028F084E603C0882319F081508093E00612
:103BF0004217530770F58091E00681508093E006EC
:103C0000241B350B2630310558F08A3010F4109201
:103C1000E0068091E0068A3018F08A508093E00632
:103C200080914B06811106C0A8DC81E080938D064F
:103C300080934B0620915106309152068091880660
:103C4000909189068217930720F414DD81E0809318
:103C50007C0680918406811146C04091CB0650912C
:103C6000CC068091810690E084179507E0F5E091FD
:103C70007506F09176064E175F0729F481E0809370
:103C8000A206809394068091A206813061F560912E
:103C90004D0670914E0620915306309154066217DE
:103CA000730778F48091E006E417F50728F48F5F36
:103CB000853628F084E603C0882319F0815080936C
:103CC000E0062617370778F41092A2068091D906ED
:103CD0009091DA06821B930B9093DA068093D906B3
:103CE00081E08093840608954091820620914F06DA
:103CF00030915006429FC001439F900D11246AE00D
:103D000070E00E94C7437093A7066093A606809157
:103D10009206853618F084E68093920690918F067D
:103D200080919206981710F49093920680919306D2
:103D30002091A3063091A40681110DC026393105CA
:103D400020F484E68093920606C02639310519F0E6
:103D500081E080939306809193064091960650915E
:103D600097068130D9F464177507C0F480919206E4
:103D70002617370770F48F5F981718F08093920614
:103D800002C09093920680919206853638F084E6C0
:103D900003C0882319F08150809392064617570775
:103DA00068F52417350770F4809192068F5F853689
:103DB00008F084E68093920680919206981710F49A
:103DC0009093920642175307C8F480919206882375
:103DD00019F0815080939206C901841B950B0B97B3
:103DE00068F0809192068A3010F4109292068091C9
:103DF00092068A3018F08A5080939206809190063D
:103E00009091E006891710F48093E006421753075B
:103E100040F48091E0068F5F853608F084E6809359
:103E2000E00608954091820620914F063091500699
:103E3000429FC001439F900D11246AE070E00E94F0
:103E4000C7437093A7066093A606809192068536B5
:103E500018F084E68093920690918F0680919206E6
:103E6000981710F49093920680919306811111C0D7
:103E70002091A3063091A4062639310520F484E66A
:103E80008093920606C02639310519F081E08093AF
:103E90009306809193064091960650919706813043
:103EA000F9F464177507E0F42091A3063091A40695
:103EB000809192062617370770F48F5F981718F0D5
:103EC0008093920602C09093920680919206853666
:103ED00038F084E603C0882319F08150809392065D
:103EE0004617570788F52091A3063091A40624179A
:103EF000350770F4809192068F5F853608F084E66E
:103F00008093920680919206981710F490939206EF
:103F100042175307C8F480919206882319F0815004
:103F200080939206241B350B2B30310568F080916D
:103F300092068A3010F410929206809192068A308E
:103F400018F08A508093920608958091750690919A
:103F500076068B35910510F01092920680919306AB
:103F6000811112C08091A3069091A406883C91050E
:103F700020F484E68093920607C0883C910521F0E6
:103F8000E5DA81E08093930680919306813081F495
:103F90008091A3069091A406813A910518F01092A1
:103FA000920608958837910518F48AE08093920666
:103FB0000895CF93C091AA06C130D9F480918706A5
:103FC000811117C08091810690E020917506309193
:103FD00076062817390768F08091A3069091A40609
:103FE0008A5591099093490680934806AFDAC093A9
:103FF00087064091820620914F0630915006429FDD
:10400000C001439F900D11246AE070E00E94C743F5
:104010007093A7066093A60680919206853618F0E5
:1040200084E68093920680919306811112C080915C
:10403000A3069091A4068C3221E0920720F484E636
:104040008093920606C08C32914019F081E08093F3
:10405000930680919306C09187068130A1F5C11126
:1040600024C0809196069091970668177907E8F426
:104070002091A3063091A406809192062617370757
:1040800078F48F5F8093920690918F06981710F4C2
:104090009093920680919206853638F084E603C0AC
:1040A000882319F08150809392068091810690E0D8
:1040B0000A9720917506309176068217930718F4B7
:1040C00086E480939206C13091F4809148069091E5
:1040D00049060E948703C0938D06809151069091F6
:1040E0005206CD9720F01092520610925106809100
:1040F0009606909197062091A6063091A706821702
:10410000930748F42091AA06211105C08A55910908
:10411000CF910C948703CF910895BC9A8091E006CB
:10412000880F81BF139A80919206880F8093860032
:1041300080917D06811102C03CDFF9DB80917D0614
:10414000813019F410929206ECDC80917D06823069
:1041500019F41092E0062DDF80917D06833011F472
:104160000E94CB0380917D06843009F4BDDD8091EF
:104170007D06853009F4B8DD80917D06863009F42E
:1041800051DE80917D06873009F4DFDE80917D0667
:10419000893069F48091A3069091A4060E944C0393
:1041A00080919206863518F081E080937C06089510
:1041B00063EC70E08CEB92E00E94194762EC71E0D6
:1041C0008EEB92E00E94194766E170E080EC92E08D
:1041D0000E94194766E170E082EC92E00E94194764
:1041E00061E070E084EC92E00E941947A8956EE6C9
:1041F00070E086EC92E00E94194764E670E088EC7B
:1042000092E00E94194764E670E08AEC92E00E9416
:10421000194760E070E08CEC92E00E941947A89585
:1042200060E070E08EEC92E00E94194760E070E080
:1042300080ED92E00E94194760E070E082ED92E02C
:104240000E94194760E070E084ED92E00E941947F7
:1042500060E070E086ED92E00E94194760E070E057
:1042600088ED92E00E941947A89566EE70E08EE90D
:1042700092E00E94194762EC71E080EA92E00E94AD
:10428000194766E170E082EA92E00E94194766E110
:1042900070E084EA92E00E94194761E070E086EAEB
:1042A00092E00E941947A89563E770E088EA92E0DF
:1042B0000E94194764E670E08AEA92E00E9419477A
:1042C00064E670E08CEA92E00E94194760E070E0DA
:1042D0008EEA92E00E94194760E070E080EB92E085
:1042E0000E94194760E070E082EB92E00E9419475B
:1042F000A89560E070E084EB92E00E94194760E0CE
:1043000070E086EB92E00E94194760E070E088EB75
:1043100092E00E94194760E070E08AEB92E00E9410
:104320001947A89566EE70E080E892E00E94194770
:1043300062EC71E082E892E00E94194766E170E069
:1043400084E892E00E94194766E170E086E892E016
:104350000E94194761E070E088E892E00E941947E6
:10436000A89563E770E08AE892E00E94194764E646
:1043700070E08CE892E00E94194764E670E08EE8F5
:1043800092E00E94194760E070E080E992E00E94AC
:10439000194760E070E082E992E00E94194760E00E
:1043A00070E084E992E00E941947A89560E070E00F
:1043B00086E992E00E94194760E070E088E992E0A7
:1043C0000E94194760E070E08AE992E00E94194774
:1043D00060E070E08CE992E00E941947A89566E9D8
:1043E00070E082E692E00E94194768EC70E084E693
:1043F00092E00E94194766E170E086E692E00E9432
:10440000194766E170E088E692E00E94194761E092
:1044100070E08AE692E00E941947A89563E770E091
:104420008CE692E00E94194764E670E08EE692E026
:104430000E94194764E670E080E792E00E94194705
:1044400060E070E082E792E00E94194760E070E06F
:1044500084E792E00E94194760E070E086E792E00E
:104460000E941947A89560E070E088E792E00E94FA
:10447000194760E070E08AE792E00E94194760E027
:1044800070E08CE792E00E94194760E070E08EE7F0
:1044900092E00E941947A8956EEB70E084E492E0E8
:1044A0000E94194768EC70E086E492E00E94194788
:1044B00066E170E088E492E00E94194766E170E0EE
:1044C0008AE492E00E94194761E070E08CE492E097
:1044D0000E941947A89564E670E08EE492E00E947D
:1044E000194764E670E080E592E00E94194764E6AF
:1044F00070E082E592E00E94194760E070E084E598
:1045000092E00E94194760E070E086E592E00E9428
:10451000194760E070E088E592E00E941947A8958D
:1045200060E070E08AE592E00E94194760E070E088
:104530008CE592E00E94194760E070E08EE592E021
:104540000E94194760E070E080E692E00E941947FF
:10455000A89566EE70E086E292E00E94194762EC50
:1045600071E088E292E00E94194766E170E08AE219
:1045700092E00E94194766E170E08CE292E00E94AE
:10458000194761E070E08EE292E00E941947A89519
:1045900063E770E080E392E00E94194764E670E010
:1045A00082E392E00E94194764E670E084E392E0BF
:1045B0000E94194760E070E086E392E00E9419478C
:1045C00060E070E088E392E00E94194760E070E0EC
:1045D0008AE392E00E941947A89560E070E08CE3BE
:1045E00092E00E94194760E070E08EE392E00E9442
:1045F000194760E070E080E492E00E94194760E0B3
:1046000070E082E492E00E941947A89566EE70E09F
:1046100088E092E00E94194762EC71E08AE092E043
:104620000E94194766E170E08CE092E00E94194711
:1046300066E170E08EE092E00E94194761E070E070
:1046400080E192E00E941947A89563E770E082E15B
:1046500092E00E94194764E670E084E192E00E94D3
:10466000194764E670E086E192E00E94194760E035
:1046700070E088E192E00E94194760E070E08AE112
:1046800092E00E94194760E070E08CE192E00E94A5
:104690001947A89560E070E08EE192E00E9419470A
:1046A00060E070E080E292E00E94194760E070E014
:1046B00082E292E00E94194760E070E084E292E0BA
:1046C0000E941947A89563EC70E08CEC91E00E9481
:1046D000194766E170E080ED91E00E94194761E0C2
:1046E00070E084ED91E00E9419476FE070E086ED84
:1046F00091E00E941947A89564E670E088ED91E08A
:104700000E94194761E070E082EE91E00E94194733
:1047100063EC70E084EE91E00E9419476AE070E07B
:1047200086EE91E00E941947A89562EC71E084E75B
:1047300091E00E94194766E170E088E791E00E94ED
:10474000194761E070E08AE791E00E9419476EE640
:1047500070E08CE791E00E941947A89564E670E04C
:1047600080E891E00E94194762E070E088E891E0FB
:104770000E94194762EC71E08AE191E00E941947BA
:1047800066E170E08CE191E00E94194762E170E01F
:104790008EE191E00E941947A89564E670E084E2FA
:1047A00091E00E94194764E670E086E291E00E9481
:1047B000194764E070E08EE291E00E9419476CE2D4
:1047C00071E084E391E00E941947A89562EC71E0E2
:1047D00080EC90E00E94194766E170E082EC90E086
:1047E0000E94194766E170E084EC90E00E9419474E
:1047F00061E070E086EC90E00E941947A8956EE6B3
:1048000070E088EC90E00E94194764E670E08AEC62
:1048100090E00E94194764E670E08CEC90E00E9402
:10482000194765E070E084ED90E00E941947A89573
:1048300062EC71E086E690E00E94194766E170E064
:104840008AE690E00E94194761E070E08CE690E013
:104850000E9419476EE670E08EE690E00E941947CC
:10486000A89564E670E082E790E00E94194766E050
:1048700070E08AE790E00E94194763EC70E08CEBEF
:1048800092E00E941947A89508956FE070E080EECD
:1048900092E00E9419476FE070E08EED92E00E9476
:1048A00019476FE070E08CED92E00E94194761E0DB
:1048B0008BED92E00E940C4761E08AED92E00C944F
:1048C0000C478FB9779BFECF8FB10895CF93A39AF2
:1048D000AB9AAB9880E0F5DFC82F80E0F2DFAB9AAF
:1048E0006C2F70E0762F6627682B687F7F7723E038
:1048F000769567952A95E1F780E090E00E94D64290
:1049000020E030E040E85EE30E943C430E94AA427F
:104910007093760660937506CB01CF910895CF937F
:10492000A79AAF9AAF9880E0CCDFC82F80E0C9DFAC
:10493000AF9A6C2F70E0762F6627682B687F7F77A1
:1049400023E0769567952A95E1F780E090E00E9454
:10495000D64220E030E040E85EE30E943C430E9403
:10496000AA427093A4066093A306CB01CF91089549
:1049700086E291E09093E9068093E80680917606BE
:104980008F93809175068F9383E092E09F938F932E
:104990000E9416448DE08A95F1F700008091500640
:1049A0008F9380914F068F938DE092E09F938F932A
:1049B0000E9416449DE09A95F1F7000080919206BE
:1049C0001F928F9387E192E09F938F930E941644EA
:1049D0008DE08A95F1F700008091E0061F928F9399
:1049E00082E292E09F938F930E9416449DE09A95F5
:1049F000F1F700008CE292E09F938F930E9416449F
:104A00008DE08A95F1F700008091A4068F93809144
:104A1000A3068F9384E392E09F938F930E941644A2
:104A2000A8958DB79EB746960FB6F8949EBF0FBE59
:104A30008DBF80917C06811108C08DE392E09F9329
:104A40008F930E9416440F900F90A89580917C063A
:104A5000813041F484E492E09F938F930E94164446
:104A60000F900F909DE09A95F1F70000E0917D0680
:104A70008E2F90E08830910508F09DC0FC01EE5823
:104A8000FF4F0C94DB438BE492E09F938F930E9443
:104A90001644A8950F900F90E091D5068E2F90E0C8
:104AA0008830910508F087C0FC01E658FF4F0C9450
:104AB000DB438AE592E071C08AE692E06EC082EA4A
:104AC00092E06BC081EB92E068C080EC92E065C040
:104AD0008FEC92E09F938F930E941644A8950F90BD
:104AE0000F9080918306813009F452C008F44DC0C4
:104AF000823009F450C008958FED92E09F938F9318
:104B00000E941644A8950F900F9080918A068130DC
:104B100009F43EC0D0F1823009F43DC0089580EF21
:104B200092E042C08EEF92E09F938F930E941644D2
:104B3000A8950F900F908091DF06813049F128F100
:104B4000823049F108958FE093E09F938F930E9404
:104B50001644A8950F900F908091D4068130C1F033
:104B6000A0F08230C1F0089582E293E09F938F938A
:104B70000E941644A8950F900F908091D106813025
:104B800039F018F0823039F0089585E792E005C0D9
:104B900084E892E002C083E992E09F938F930E94A1
:104BA000164407C084E393E09F938F930E941644BA
:104BB000A8950F900F900895CF92DF92EF92FF92F9
:104BC0000F931F93CF93DF9300D000D0CDB7DEB704
:104BD00080917C06813009F034C180918B069091E0
:104BE0008C06892BD9F40FE110E024E230E04AE58D
:104BF00050E064E670E088E090E00E94CD0A24E294
:104C000030E04AE550E064E670E08FED90E00E940D
:104C1000CD0AA895A49AAC980E944612CC24C394BD
:104C2000D12C80917C06813009F00BC1A895A0DEC3
:104C30008091D7069091D8068A35910549F42FEFD7
:104C40008DE399E4215080409040E1F700C00000DE
:104C5000A89503E02FE130E04FEF5FEF69E170E0EE
:104C600085E890E00E947D198091630080FD81C0FD
:104C7000A8951C821B821A821982BE016F5F7F4F2A
:104C8000CE0103960E943E428B819C8184319540E7
:104C900088F489819A81883D9E4060F489819A8157
:104CA000853C994038F0D0928C06C0928B061092C9
:104CB0009A0613D48B819C818431954098F5898123
:104CC0009A818C3D954070F589819A81853F91400C
:104CD00048F1D0928C06C0928B061092AB06809160
:104CE0007D06811102C00E94E03780917D068130EF
:104CF00011F40E94CC3A80917D06823011F40E941A
:104D0000D33B80917D06843011F40E94DA3C80917F
:104D10007D06853009F4ADD480917D06863011F48E
:104D20000E94D83680914106813019F58B819C8193
:104D3000853C9940F0F089819A818C3D9540C8F47A
:104D400089819A81853F9140A0F0D0928C06C092D3
:104D50008B060E94041A80E00E94E5400E944F41A9
:104D600010928C0610928B068FE190E00E94420C0C
:104D700023DFACDD0E94D317A8958FEF91EE24E0DE
:104D8000815090402040E1F700C00000C8DDA895A8
:104D90000E945518E0909206F12C02E02FE130E0DD
:104DA0004FEF5FEF6EE670E08CE190E00E94080C40
:104DB000E090E006F12C2FE130E04FEF5FEF6EE680
:104DC00070E080EF90E00E94080C809141068130F5
:104DD00011F40E94D7410E947C1180917C068111C0
:104DE00020CFA8950E94511BA8950E94A61AA895AD
:104DF0000E9446120FE110E029E130E04AE550E060
:104E00006EE670E088E090E00E94CD0A29E130E093
:104E10004AE550E06EE670E08FED90E00E94CD0A2A
:104E200080914106813021F40E94E0400E940E42B0
:104E30001092500610924F0610928C0610928B061C
:104E4000F0CE0F900F900F900F90DF91CF911F91A8
:104E50000F91FF90EF90DF90CF900895EF92FF9227
:104E60000F931F93CF93DF9380919906813009F0C0
:104E700047C18FE190E00E94420C0E948B1485E0B4
:104E800080939F06C5E080919906813009F038C172
:104E90000E94CF1580919F068230D9F48091CA0676
:104EA0008F5F8093CA060FE110E02CE330E046EEFE
:104EB00050E069E670E081E090E00E94CD0A22E3D4
:104EC00030E043EC50E068E270E088E090E00E945F
:104ED000CD0A80919F068330D9F48091CA06815013
:104EE0008093CA060FE110E02CE330E046EE50E07C
:104EF00069E670E081E090E00E94CD0A22E330E0B4
:104F000043EC50E068E270E088E090E00E94CD0A57
:104F10008091CA06853010F01092CA068091CA06A8
:104F2000823081F1B8F48823D9F0813009F0C1C012
:104F300070E0E72E76E0F72E01E02FE130E04FEF52
:104F40005FEF6CE370E088E090E00E94C20B8EEDB2
:104F500092E029C08330B1F1843009F471C0A9C056
:104F6000E9E1EE2EE6E0FE2E01E02FE130E04FEF2A
:104F70005FEF6CE370E08FE090E00E94C20B80EE88
:104F800092E011C064EFE62E65E0F62E01E02FE11D
:104F900030E04FEF5FEF6CE370E082E390E00E945F
:104FA000C20B8CED92E00E94FE467C0103E02FE1F3
:104FB00030E04FEF5FEF62E870E080E590E00E9444
:104FC000080C77C04CEDE42E45E0F42E01E02FE113
:104FD00030E04FEF5FEF6CE370E088E290E00E941A
:104FE000C20B5AEEE52E55E0F52E02E02FE130E03F
:104FF0004FEF5FEF62E870E088E290E00E94C20B42
:1050000080919F06811119C0D3D83FDC36EAE32E88
:1050100035E0F32E2FE130E04FEF5FEF62E870E014
:1050200088E290E00E94C20B2FEF89E698E12150C0
:1050300080409040E1F700C00000C0939F0639C057
:105040002BECE22E25E0F22E01E02FE130E04FEFD5
:105050005FEF6CE370E08EE190E00E94C20B8BED9D
:1050600092E00E94F646813079F49DEBE92E95E0BE
:10507000F92E03E02FE130E04FEF5FEF62E870E0E0
:1050800080E590E00E94C20B8BED92E00E94F64614
:1050900081110FC088EBE82E85E0F82E03E02FE1A8
:1050A00030E04FEF5FEF62E870E080E590E00E9453
:1050B000C20BD0919F06D13069F4109299061092DC
:1050C0008C0610928B068FE190E00E94420CD093E8
:1050D0007C0672DD80919F06811106C081E080937D
:1050E00099061092DC0613D0C0939F062FE785EB3C
:1050F00091E0215080409040E1F700C00000C3CE15
:10510000DF91CF911F910F91FF90EF900895BF9283
:10511000CF92DF92EF92FF920F931F93CF93DF9383
:105120008091DC068111CFC185E080939F06C9E1A3
:10513000D0E025E0C22ED12C35E0B32E8091DC06E4
:105140008111C1C18091CA06813009F46FC038F065
:10515000823009F4DDC0843009F441C1A4C180EE7D
:1051600092E00E94FE467C0103E02FE130E040E047
:1051700058EF62E870E080E590E00E94080C80EE55
:1051800092E00E94FE4690939E0680939D060E94A8
:10519000CF1580919F068230A9F480919D06909151
:1051A0009E06019690939E0680939D060FE110E067
:1051B0002CE330E046EE50E069E670E081E090E0FC
:1051C0000E94CD0A80919F068330A9F480919D06AC
:1051D00090919E06019790939E0680939D060FE105
:1051E00010E02CE330E046EE50E069E670E081E04C
:1051F00090E00E94CD0A80919D0690919E064A976C
:1052000020F0D0939E06C0939D0680919D069091BC
:105210009E060A9720F4D0939E06C0939D06609147
:105220009D0670919E0680EE92E066C08EED92E043
:105230000E94FE467C0103E02FE130E040E058EFA1
:1052400062E870E080E590E00E94080C8EED92E04C
:105250000E94FE469093800680937F060E94CF15A1
:1052600080919F068230A9F480917F0690918006FC
:1052700001969093800680937F060FE110E02CE367
:1052800030E046EE50E069E670E081E090E00E9498
:10529000CD0A80919F068330A9F480917F0690917A
:1052A000800601979093800680937F060FE110E0BF
:1052B0002CE330E046EE50E069E670E081E090E0FB
:1052C0000E94CD0A80917F06909180064A9720F037
:1052D000D0938006C0937F0680917F0690918006D0
:1052E0000A9720F4D0938006C0937F0660917F06D2
:1052F000709180068EED92E00E9419472FE788E3B7
:1053000091E0215080409040E1F700C00000CBC008
:105310008CED92E00E94FE467C0103E02FE130E03C
:1053200040E058EF62E870E080E590E00E94080CF1
:105330008CED92E00E94FE4690939C0680939B0623
:105340000E94CF1580919F068230A9F480919B0620
:1053500090919C06019690939C0680939B060FE18A
:1053600010E02CE330E046EE50E069E670E081E0CA
:1053700090E00E94CD0A80919F068330A9F480912D
:105380009B0690919C06019790939C0680939B06A8
:105390000FE110E02CE330E046EE50E069E670E00B
:1053A00081E090E00E94CD0A80919B0690919C063E
:1053B0004F9720F0D0929C06C0929B0680919B064E
:1053C00090919C06059720F4D0929C06C0929B0673
:1053D00060919B0670919C068CED92E08DCF8BEDD9
:1053E00092E00E94F646809343060E94CF1580917A
:1053F0009F06823089F4809143068F5F8093430635
:105400000FE110E02CE330E046EE50E069E670E09A
:1054100081E090E00E94CD0A80919F06833089F45C
:10542000809143068150809343060FE110E02CE306
:1054300030E046EE50E069E670E081E090E00E94E6
:10544000CD0A80914306823010F01092430680917D
:105450004306813079F49DEBE92E95E0F92E03E0C7
:105460002FE130E040E058EF62E870E080E590E046
:105470000E94C20B8091430681110FC088EBE82E79
:1054800085E0F82E03E02FE130E040E058EF62E8DD
:1054900070E080E590E00E94C20B609143068BEDC6
:1054A00092E00E940C4780919F06813049F48093DE
:1054B000DC06809399068FE190E00E94420CCEDCDE
:1054C000B0929F063BCEDF91CF911F910F91FF903D
:1054D000EF90DF90CF90BF9008959F92AF92BF92D0
:1054E000CF92DF92EF92FF920F931F93CF93DF93B0
:1054F00080919A068111B1C08FE190E00E94420C28
:105500000E94FA1385E080939F0610929906C0E0EE
:1055100089E0E82ED1E097E0D92E26E0C22E35E0D2
:10552000F32E44E0B42E53E0A52E62E0962E809137
:105530009A06811192C00E94CF1580919F068230F9
:1055400069F4CF5F0FE110E02CE330E046EE50E06D
:1055500069E670E081E090E00E94CD0A80919F06AC
:10556000833069F4C1500FE110E02CE330E046EEE7
:1055700050E069E670E081E090E00E94CD0ACA3018
:1055800008F0C0E08C2F0E94FB128C2F90E08A3034
:105590009105A0F5FC01EE57FF4F0C94DB431092F0
:1055A000990610927D062AC010929906D0937D0626
:1055B00025C01092990690927D0620C010929906FF
:1055C000A0927D061BC010929906B0927D0616C06F
:1055D00010929906F0927D0611C010929906C09221
:1055E0007D060CC010929906D0927D0607C0D0931C
:1055F000990604C010929906E0927D0680919F065C
:105600008130F9F480919906813049F410927D0639
:1056100010929A068FE190E00E94420C1FDCD0931A
:105620009A0610928C0610928B0680917D0690E06F
:1056300090936C0680936B068FE190E00E94420C81
:10564000BBDAF0929F062FEF80E792E02150804076
:105650009040E1F700C000006ACFDF91CF911F9129
:105660000F91FF90EF90DF90CF90BF90AF909F9001
:105670000895EF92FF920F931F93CF93DF93A89516
:105680008091AB068111F4C08FE190E00E94420C42
:105690000E943E158091D40690E0909386068093F8
:1056A000850685E080939F06C1E0D5E08091AB063A
:1056B0008111DEC0A8950E94CF1580919F0682308F
:1056C000A9F48091850690918606019690938606AE
:1056D000809385060FE110E02CE330E046EE50E0C9
:1056E00069E670E081E090E00E94CD0A80919F061B
:1056F0008330A9F480918506909186060197909356
:105700008606809385060FE110E02CE330E046EE3C
:1057100050E069E670E081E090E00E94CD0A80915F
:10572000850690918606039720F0109286061092C7
:10573000850680918506909186068130910589F1D4
:10574000D0F0029709F046C08EE7E82E85E0F82EEB
:1057500002E02FE130E04FEF5FEF6DE770E088E2AD
:1057600090E00E94C20B82E08093D4064EE150E0AC
:1057700062E870E02BC022E9E22E25E0F22E02E082
:105780002FE130E04FEF5FEF6DE770E088E290E0EF
:105790000E94C20B1092D4064EE150E06EEB70E016
:1057A00015C098E8E92E95E0F92E02E02FE130E0EF
:1057B0004FEF5FEF6DE770E088E290E00E94C20B70
:1057C000C093D4064EE150E060EA70E085E596E0D3
:1057D0000E94E64680919F0681110FC0A895C09354
:1057E000AB0610928C0610928B06C0939A068FE13E
:1057F00090E00E94420CA895DFD980919F068130ED
:1058000059F5A8958093AB0610928C0610928B06E2
:1058100080939A068FE190E00E94420CA895109226
:10582000E1068091D406813069F038F0823091F43D
:105830004EE150E062E870E009C04EE150E06EEBEE
:1058400070E004C04EE150E060EA70E085E596E06B
:105850000E94E646A89513D0D0939F062FEF80E7CD
:1058600092E0215080409040E1F700C000001ECF40
:10587000DF91CF911F910F91FF90EF900895EF92DC
:10588000FF920F931F93CF938091E10681110C94A7
:10589000D2368FE190E00E94420C0E94391685E0DA
:1058A00080939F06C5E08091E10681110C94D23669
:1058B0000E94CF1580919F068230D9F48091D00646
:1058C0008F5F8093D0060FE110E02CE330E046EECE
:1058D00050E069E670E081E090E00E94CD0A22E3AA
:1058E00030E043EC50E068E270E088E090E00E9435
:1058F000CD0A80919F068330D9F48091D0068150E3
:105900008093D0060FE110E02CE330E046EE50E04B
:1059100069E670E081E090E00E94CD0A22E330E089
:1059200043EC50E068E270E088E090E00E94CD0A2D
:105930008091D0068E3010F01092D006E091D00603
:105940008E2F90E08E30910510F00C948D35FC0177
:10595000E457FF4F80917D060C94DB43811137C0E3
:105960008091550690915606893E934020F0109202
:1059700056061092550670E3E72E75E0F72E01E00B
:105980002FE130E04FEF5FEF62E370E08FE090E0F7
:105990000E94C20BE9E2EE2EE5E0FE2E2FE130E0A0
:1059A0004FEF5FEF66E470E08CE390E00E94C20B83
:1059B000E0905506F090560603E02FE130E04FEFFF
:1059C0005FEF62E870E080E590E00E94080C809153
:1059D0007D06813009F0B6C7809155069091560634
:1059E000893E934020F0109256061092550650E3DF
:1059F000E52E55E0F52E01E02FE130E04FEF5FEFAF
:105A000062E370E08FE090E00E94C20B69E2E62E54
:105A100065E0F62E2FE130E04FEF5FEF66E470E0D7
:105A20008CE390E00E94C20BE0905506F090560681
:105A30007EC7811137C08091570690915806893EE4
:105A4000934020F0109258061092570631E1E32E51
:105A500035E0F32E01E02FE130E04FEF5FEF62E33E
:105A600070E08FE090E00E94C20B43E0E42E45E03E
:105A7000F42E2FE130E04FEF5FEF66E470E08CE34F
:105A800090E00E94C20BE0905706F090580603E0A9
:105A90002FE130E04FEF5FEF62E870E080E590E0EB
:105AA0000E94080C80917D06813031F48091D006EF
:105AB0008F5F8093D00639C08230B9F58091570648
:105AC00090915806893E934020F01092580610920B
:105AD000570691E1E92E95E0F92E01E02FE130E043
:105AE0004FEF5FEF62E370E08FE090E00E94C20B47
:105AF00023E0E22E25E0F22E2FE130E04FEF5FEFC2
:105B000066E470E08CE390E00E94C20BE0905706E0
:105B1000F090580603E02FE130E04FEF5FEF62E8CE
:105B200070E080E590E00E94080C80917D06843052
:105B3000B9F58091570690915806893E934020F020
:105B4000109258061092570601E1E02E05E0F02E63
:105B500001E02FE130E04FEF5FEF62E370E08FE0B4
:105B600090E00E94C20B83E0E82E85E0F82E2FE142
:105B700030E04FEF5FEF66E470E08CE390E00E946E
:105B8000C20BE0905706F090580603E02FE130E09A
:105B90004FEF5FEF62E870E080E590E00E94080C54
:105BA00080917D068530B9F5809157069091580611
:105BB000893E934020F01092580610925706B1E1AA
:105BC000EB2EB5E0FB2E01E02FE130E04FEF5FEF71
:105BD00062E370E08FE090E00E94C20B13E0E12EE0
:105BE00015E0F12E2FE130E04FEF5FEF66E470E05B
:105BF0008CE390E00E94C20BE0905706F0905806AC
:105C000003E02FE130E04FEF5FEF62E870E080E506
:105C100090E00E94080C80917D06863009F07DC7D7
:105C20008091570690915806893E934020F010923B
:105C3000580610925706F1E1EF2EF5E0FF2E01E035
:105C40002FE130E04FEF5FEF62E370E08FE090E034
:105C50000E94C20BA3E0EA2EA5E0FA2E2FE130E06D
:105C60004FEF5FEF66E470E08CE390E00E94C20BC0
:105C7000E0905706F0905806B2C5811136C0809169
:105C8000590690915A064F9720F010925A0610929A
:105C900059067BEEE72E74E0F72E01E02FE130E0AD
:105CA0004FEF5FEF62E370E08FE090E00E94C20B85
:105CB000E3EDEE2EE4E0FE2E2FE130E04FEF5FEF5C
:105CC00066E470E08FE090E00E94C20BE09059061D
:105CD000F0905A0603E02FE130E04FEF5FEF62E80B
:105CE00070E080E590E00E94080C80917D06813094
:105CF00009F028C68091590690915A064F9720F0D6
:105D000010925A06109259065BEEE52E54E0F52EDD
:105D100001E02FE130E04FEF5FEF62E370E08FE0F2
:105D200090E00E94C20B63EDE62E64E0F62E2FE1B8
:105D300030E04FEF5FEF66E470E08FE090E00E94AC
:105D4000C20BE0905906F0905A06F1C5811136C099
:105D500080915B0690915C064F9720F010925C0654
:105D600010925B063BEBE32E34E0F32E01E02FE1D3
:105D700030E04FEF5FEF62E370E08FE090E00E9471
:105D8000C20B43EAE42E44E0F42E2FE130E04FEF63
:105D90005FEF66E470E08FE090E00E94C20BE0905D
:105DA0005B06F0905C0603E02FE130E04FEF5FEF21
:105DB00062E870E080E590E00E94080C80917D062A
:105DC000813031F48091D0068F5F8093D00638C047
:105DD0008230B1F580915B0690915C064F9720F080
:105DE00010925C0610925B069BEBE92E94E0F92E74
:105DF00001E02FE130E04FEF5FEF62E370E08FE012
:105E000090E00E94C20B23EAE22E24E0F22E2FE162
:105E100030E04FEF5FEF66E470E08FE090E00E94CB
:105E2000C20BE0905B06F0905C0603E02FE130E0EF
:105E30004FEF5FEF62E870E080E590E00E94080CB1
:105E400080917D068430B1F580915B0690915C066F
:105E50004F9720F010925C0610925B060BEBE02E41
:105E600004E0F02E01E02FE130E04FEF5FEF62E35E
:105E700070E08FE090E00E94C20B83EAE82E84E09D
:105E8000F82E2FE130E04FEF5FEF66E470E08FE037
:105E900090E00E94C20BE0905B06F0905C0603E08D
:105EA0002FE130E04FEF5FEF62E870E080E590E0D7
:105EB0000E94080C80917D068530B1F580915B06CB
:105EC00090915C064F9720F010925C0610925B0652
:105ED000BBEBEB2EB4E0FB2E01E02FE130E04FEF07
:105EE0005FEF62E370E08FE090E00E94C20B13EA84
:105EF000E12E14E0F12E2FE130E04FEF5FEF66E48A
:105F000070E08FE090E00E94C20BE0905B06F090A2
:105F10005C0603E02FE130E04FEF5FEF62E870E0F6
:105F200080E590E00E94080C80917D06863009F0A3
:105F3000F4C580915B0690915C064F9720F010921B
:105F40005C0610925B06FBEBEF2EF4E0FF2E01E007
:105F50002FE130E04FEF5FEF62E370E08FE090E021
:105F60000E94C20BA3EAEA2EA4E0FA2E2FE130E051
:105F70004FEF5FEF66E470E08FE090E00E94C20BAD
:105F8000E0905B06F0905C062AC4811145C08091C8
:105F90005D0690915E06039730F081E090E090936B
:105FA0005E0680935D06EBE8EE2EE4E0FE2E01E057
:105FB0002FE130E04FEF5FEF6CE370E08FE090E0B7
:105FC0000E94C20B80915D0690915E06019779F464
:105FD0007DEBE72E75E0F72E03E02FE130E04FEF89
:105FE0005FEF62E870E080E590E00E94C20B809174
:105FF0005D0690915E06892B79F468EBE62E65E0EC
:10600000F62E03E02FE130E04FEF5FEF62E870E043
:1060100080E590E00E94C20B80917D06813009F0FE
:1060200045C080915D0690915E06039730F081E057
:1060300090E090935E0680935D065BE8E52E54E069
:10604000F52E01E02FE130E04FEF5FEF6CE370E001
:106050008FE090E00E94C20B80915D0690915E06F9
:10606000019779F44DEBE42E45E0F42E03E02FE1A7
:1060700030E04FEF5FEF62E870E080E590E00E9473
:10608000C20B80915D0690915E06892B79F438EB06
:10609000E32E35E0F32E03E02FE130E04FEF5FEF2A
:1060A00062E870E080E590E00E94C20B80917D067E
:1060B000823009F045C080915D0690915E0603979D
:1060C00030F081E090E090935E0680935D062BE8CF
:1060D000E22E24E0F22E01E02FE130E04FEF5FEFFF
:1060E0006CE370E08FE090E00E94C20B80915D064F
:1060F00090915E06019779F49DEBE92E95E0F92EDB
:1061000003E02FE130E04FEF5FEF62E870E080E501
:1061100090E00E94C20B80915D0690915E06892BF3
:1061200079F488EBE82E85E0F82E03E02FE130E0EB
:106130004FEF5FEF62E870E080E590E00E94C20BF5
:1061400080917D069CEF980F923008F4A5C48630AC
:1061500009F0E3C480915D0690915E06039730F0EC
:1061600081E090E090935E0680935D060BE8E02E60
:1061700004E0F02E01E02FE130E04FEF5FEF6CE341
:1061800070E08FE090E00E94C20B80915D069091DC
:106190005E06019779F41DEBE12E15E0F12E03E088
:1061A0002FE130E04FEF5FEF62E870E080E590E0D4
:1061B0000E94C20B80915D0690915E06892B09F0CA
:1061C000ACC4B8EBEB2EB5E0FB2E03E02FE130E0E2
:1061D0004FEF5FEF62E870E080E590E00E94C20B55
:1061E0009CC4811137C080915F06909160068F3505
:1061F000914020F01092600610925F06F3E7EF2EB8
:10620000F4E0FF2E01E02FE130E04FEF5FEF62E3BB
:1062100070E08FE090E00E94C20BABE5EA2EA4E0B4
:10622000FA2E2FE130E04FEF5FEF66E470E08FE091
:1062300090E00E94C20BE0905F06F090600603E0E1
:106240002FE130E04FEF5FEF62E870E080E590E033
:106250000E94080C80917D068130B9F580915F061F
:10626000909160068F35914020F010926006109258
:106270005F0673E7E72E74E0F72E01E02FE130E0D0
:106280004FEF5FEF62E370E08FE090E00E94C20B9F
:10629000EBE5EE2EE4E0FE2E2FE130E04FEF5FEF76
:1062A00066E470E08FE090E00E94C20BE0905F0631
:1062B000F090600603E02FE130E04FEF5FEF62E81F
:1062C00070E080E590E00E94080C80917D068230AD
:1062D000B9F580915F06909160068F35914020F06E
:1062E0001092600610925F0653E7E52E54E0F52EFB
:1062F00001E02FE130E04FEF5FEF62E370E08FE00D
:1063000090E00E94C20B6BE5E62E64E0F62E2FE1D2
:1063100030E04FEF5FEF66E470E08FE090E00E94C6
:10632000C20BE0905F06F090600603E02FE130E0E2
:106330004FEF5FEF62E870E080E590E00E94080CAC
:1063400080917D069CEF980F923008F4A5C38630AB
:1063500009F0E3C380915F06909160068F3591400C
:1063600020F01092600610925F0633E7E32E34E0CF
:10637000F32E01E02FE130E04FEF5FEF62E370E0DA
:106380008FE090E00E94C20B4BE5E42E44E0F42E37
:106390002FE130E04FEF5FEF66E470E08FE090E0D8
:1063A0000E94C20BE0905F06F090600618C2811157
:1063B00037C080916106909162068636910520F083
:1063C000109262061092610693E4E92E94E0F92E91
:1063D00001E02FE130E04FEF5FEF62E370E08FE02C
:1063E00090E00E94C20B2BE2E22E24E0F22E2FE17D
:1063F00030E04FEF5FEF66E470E08FE090E00E94E6
:10640000C20BE0906106F090620603E02FE130E0FD
:106410004FEF5FEF62E870E080E590E00E94080CCB
:1064200080917D068130B9F5809161069091620678
:106430008636910520F0109262061092610603E400
:10644000E02E04E0F02E01E02FE130E04FEF5FEFAF
:1064500062E370E08FE090E00E94C20B8BE2E82ED6
:1064600084E0F82E2FE130E04FEF5FEF66E470E05C
:106470008FE090E00E94C20BE0906106F09062060F
:1064800003E02FE130E04FEF5FEF62E870E080E57E
:1064900090E00E94080C80917D06823031F480915A
:1064A000D0068F5F8093D00639C08430B9F58091D3
:1064B0006106909162068636910520F01092620680
:1064C00010926106B3E4EB2EB4E0FB2E01E02FE165
:1064D00030E04FEF5FEF62E370E08FE090E00E940A
:1064E000C20B1BE2E12E14E0F12E2FE130E04FEF62
:1064F0005FEF66E470E08FE090E00E94C20BE090F6
:106500006106F090620603E02FE130E04FEF5FEFAD
:1065100062E870E080E590E00E94080C80917D06C2
:106520008530B9F5809161069091620686369105B5
:1065300020F01092620610926106F3E4EF2EF4E070
:10654000FF2E01E02FE130E04FEF5FEF62E370E0FC
:106550008FE090E00E94C20BABE2EA2EA4E0FA2E9C
:106560002FE130E04FEF5FEF66E470E08FE090E006
:106570000E94C20BE0906106F090620603E02FE1FA
:1065800030E04FEF5FEF62E870E080E590E00E945E
:10659000080C80917D067DC2811137C08091630611
:1065A000909164068636910520F010926406109250
:1065B000630673E1E72E74E0F72E01E02FE130E08F
:1065C0004FEF5FEF62E370E08FE090E00E94C20B5C
:1065D000EBEFEE2EE3E0FE2E2FE130E04FEF5FEF2A
:1065E00066E470E08FE090E00E94C20BE0906306EA
:1065F000F090640603E02FE130E04FEF5FEF62E8D8
:1066000070E080E590E00E94080C80917D0681306A
:1066100031F48091D0068F5F8093D00639C08230EC
:10662000B9F580916306909164068636910520F055
:10663000109264061092630653E1E52E54E0F52EA5
:1066400001E02FE130E04FEF5FEF62E370E08FE0B9
:1066500090E00E94C20B6BEFE62E63E0F62E2FE176
:1066600030E04FEF5FEF66E470E08FE090E00E9473
:10667000C20BE0906306F090640603E02FE130E087
:106680004FEF5FEF62E870E080E590E00E94080C59
:1066900080917D068430B9F58091630690916406FF
:1066A0008636910520F0109264061092630633E15D
:1066B000E32E34E0F32E01E02FE130E04FEF5FEF07
:1066C00062E370E08FE090E00E94C20B4BEFE42E9B
:1066D00043E0F42E2FE130E04FEF5FEF66E470E02F
:1066E0008FE090E00E94C20BE0906306F090640699
:1066F00003E02FE130E04FEF5FEF62E870E080E50C
:1067000090E00E94080C80917D068530B9F580915B
:106710006306909164068636910520F01092640617
:106720001092630693E1E92E94E0F92E01E02FE147
:1067300030E04FEF5FEF62E370E08FE090E00E94A7
:10674000C20B2BEFE22E23E0F22E2FE130E04FEFD1
:106750005FEF66E470E08FE090E00E94C20BE09093
:106760006306F090640603E02FE130E04FEF5FEF47
:1067700062E870E080E590E00E94080C80917D0660
:10678000863009F0CAC1809163069091640686360E
:10679000910520F0109264061092630613E1E12E39
:1067A00014E0F12E01E02FE130E04FEF5FEF62E304
:1067B00070E08FE090E00E94C20B8BEFE82E83E048
:1067C000F82E2FE130E04FEF5FEF66E470E08FE0EE
:1067D00090E00E94C20BE0906306F090640603E034
:1067E0002FE130E04FEF5FEF62E870E080E590E08E
:1067F0000E94080C92C1811129C080916D06909170
:106800006E068D32914020F010926E0610926D0649
:10681000BBE7EB2EB3E0FB2E01E02FE130E04FEFC2
:106820005FEF6CE370E08FE090E00E94C20BE090BD
:106830006D06F0906E0603E02FE130E04FEF5FEF62
:1068400062E870E080E590E00E94080C80917D068F
:10685000813009F077C080916D0690916E068D327F
:10686000914020F010926E0610926D06ABE7EA2E72
:10687000A3E0FA2E01E02FE130E04FEF5FEF6CE391
:1068800070E08FE090E00E94C20BE0906D06F09007
:106890006E064DC0811129C080916F0690917006DF
:1068A000893E934020F01092700610926F06F1ED31
:1068B000EF2EF3E0FF2E01E02FE130E04FEF5FEF2E
:1068C0006CE370E08FE090E00E94C20BE0906F06F6
:1068D000F090700603E02FE130E04FEF5FEF62E8E9
:1068E00070E080E590E00E94080C80917D06813088
:1068F00049F580916F0690917006893E934020F093
:106900001092700610926F06E1EDEE2EE3E0FE2E7F
:1069100001E02FE130E04FEF5FEF6CE370E08FE0DC
:1069200090E00E94C20BE0906F06F090700603E0CA
:106930002FE130E04FEF5FEF62E870E080E590E03C
:106940000E94080C80917D06823009F4A5C09CEF5E
:10695000980F923008F09DC09FC0811190C0809127
:10696000650690916606039720F0109266061092D5
:10697000650679EEE72E73E0F72E01E02FE130E0B7
:106980004FEF5FEF6CE370E08EE190E00E94C20B8E
:106990008091650690916606019779F46DEBE62E7D
:1069A00065E0F62E03E02FE130E04FEF5FEF62E8A5
:1069B00070E080E590E00E94C20B809165069091A6
:1069C0006606892B79F458EBE52E55E0F52E03E0A9
:1069D0002FE130E04FEF5FEF62E870E080E590E09C
:1069E0000E94C20B809165068093420648C08111C7
:1069F00046C080914206811108C08DC081113FC000
:106A00008091420681119EC186C0813009F085C007
:106A10008091670690916806893E934020F010921D
:106A200068061092670633E7E32E34E0F32E01E0A8
:106A30002FE130E04FEF5FEF62E370E08FE090E036
:106A40000E94C20B4BEBE42E43E0F42E2FE130E02A
:106A50004FEF5FEF66E470E08FE090E00E94C20BC2
:106A6000E0906706F090680603E02FE130E04FEF1A
:106A70005FEF62E870E080E590E00E94080C809192
:106A80007D06813049F0823039F0843029F085303C
:106A900019F0863009F041C08091D0068F5F809355
:106AA000D0063BC0882321F09FEF980F923018F456
:106AB0001092D0062BC0843049F5809171069091D8
:106AC0007206893E934020F0109272061092710671
:106AD00084E5E82E83E0F82E01E02FE130E04FEF6F
:106AE0005FEF6CE370E08FE090E00E94C20BE090FB
:106AF0007106F090720603E02FE130E04FEF5FEF98
:106B000062E870E080E590E00E94080C80917D06CC
:106B10008550823010F41092D00680919F0681300B
:106B200009F0F3C08093E1061092AB0680917D06D8
:106B3000811128C0E0918506F0918606E830F105C4
:106B400008F5E656FF4F4EE150E00C94DB436CEB4A
:106B500072E014C06EE972E011C060E872E00EC02D
:106B600062E672E00BC064E472E008C066E272E0C4
:106B700005C068E072E002C06AEE71E085E596E06B
:106B80000E94034780917D068130E1F48091850663
:106B9000909186068130910569F038F0029791F462
:106BA0004EE150E060E971E009C04EE150E06CEC6C
:106BB00071E004C04EE150E06EEA71E085E596E0D8
:106BC0000E94034780917D068230E1F48091850622
:106BD000909186068130910569F038F0029791F422
:106BE0004EE150E066E371E009C04EE150E062E73B
:106BF00071E004C04EE150E064E571E085E596E0A7
:106C00000E94034780917D068430E1F480918506DF
:106C1000909186068130910569F038F0029791F4E1
:106C20004EE150E06CED70E009C04EE150E068E1EB
:106C300071E004C04EE150E06AEF70E085E596E057
:106C40000E94034780917D068530E1F4809185069E
:106C5000909186068130910569F038F0029791F4A1
:106C60004EE150E062E870E009C04EE150E06EEBAA
:106C700070E004C04EE150E060EA70E085E596E027
:106C80000E94034780917D068630E1F4809185065D
:106C9000909186068130910569F038F0029791F461
:106CA0004EE150E068E270E009C04EE150E064E679
:106CB00070E004C04EE150E066E470E085E596E0E7
:106CC0000E9403478FE190E00E94420C80917D0674
:106CD000811101C075D180917D06813009F45CD4A9
:106CE00080917D06823009F45ED580917D068430E6
:106CF00009F460D680917D06853011F40E94392B0D
:106D000080917D06863009F453D080919F068111D1
:106D10000CC081E08093E1061092AB0610927306DE
:106D20008FE190E00E94420CEED2C0939F068FE765
:106D300098E321E0815090402040E1F700C000003E
:106D40000C94532C813009F0E8CE80916906909123
:106D50006A06893E934020F010926A0610926906F6
:106D600094EAE92E93E0F92E01E02FE130E04FEFB5
:106D70005FEF62E370E08FE090E00E94C20B21E9D8
:106D8000E22E23E0F22E2FE130E04FEF5FEF66E4DA
:106D900070E08FE090E00E94C20BE0906906F090F6
:106DA0006A0662CECF911F910F91FF90EF900895E8
:106DB000EF92FF920F931F93CF93DF93A89580914B
:106DC000AB068111F6C08FE190E00E94420C0E9458
:106DD0003E158091D10690E09093860680938506BB
:106DE00085E080939F06C1E0D5E08091AB068111DC
:106DF000E0C0A8950E94CF1580919F068230A9F42B
:106E000080918506909186060196909386068093E0
:106E100085060FE110E02CE330E046EE50E069E635
:106E200070E081E090E00E94CD0A80919F0683305F
:106E3000A9F4809185069091860601979093860625
:106E4000809385060FE110E02CE330E046EE50E041
:106E500069E670E081E090E00E94CD0A80918506AD
:106E600090918606039720F0109286061092850670
:106E700080918506909186068130910589F1D0F048
:106E8000029709F046C08EE7E82E85E0F82E02E072
:106E90002FE130E04FEF5FEF6DE770E088E290E0C8
:106EA0000E94C20B82E08093D1064EE150E068E27E
:106EB00070E02BC022E9E22E25E0F22E02E02FE165
:106EC00030E04FEF5FEF6DE770E088E290E00E9406
:106ED000C20B1092D1064EE150E064E670E015C09E
:106EE00098E8E92E95E0F92E02E02FE130E04FEF2F
:106EF0005FEF6DE770E088E290E00E94C20BC09304
:106F0000D1064EE150E066E470E085E596E00E942F
:106F1000E64680919F06811110C0A895C093AB06EC
:106F200010928C0610928B06C0939A068FE190E027
:106F30000E94420CA8950E94DC2580919F0681301A
:106F400061F5A8958093AB0610928C0610928B0683
:106F500080939A068FE190E00E94420CA8951092CF
:106F6000E1068091D106813069F038F0823091F4E9
:106F70004EE150E068E270E009C04EE150E064E6A6
:106F800070E004C04EE150E066E470E085E596E014
:106F90000E94E646A8950E943F2CD0939F062FEFB3
:106FA00080E792E0215080409040E1F700C000006F
:106FB0001CCFDF91CF911F910F91FF90EF9008951B
:106FC000AF92BF92CF92DF92EF92FF920F931F93F7
:106FD000CF93DF93A8958091AB06811189C18FE192
:106FE00090E00E94420C0E943E158091D50690E0F0
:106FF000909386068093850685E080939F06E7E060
:10700000DE2EF6E0CF2ED5E0A4E0BA2EB3E0AB2E14
:10701000C1E08091AB0681116BC1A8950E94CF158C
:1070200080919F068230A9F4809185069091860612
:10703000019690938606809385060FE110E02CE37D
:1070400030E046EE50E069E670E081E090E00E94BA
:10705000CD0A80919F068330A9F480918506909196
:107060008606019790938606809385060FE110E0CF
:107070002CE330E046EE50E069E670E081E090E01D
:107080000E94CD0A8091850690918606089720F08F
:107090001092860610928506E0918506F09186068C
:1070A000E830F10508F0BEC0EE55FF4F0C94DB430D
:1070B00071EAE72E75E0F72E02E02FE130E04FEFA6
:1070C0005FEF6DE770E082E390E00E94C20B1092E8
:1070D000D5064EE150E06CEB72E09AC06CE9E62E0A
:1070E00065E0F62E02E02FE130E04FEF5FEF6DE755
:1070F00070E082E390E00E94C20BC093D5064EE19F
:1071000050E06EE972E084C052E9E52E55E0F52EBC
:1071100002E02FE130E04FEF5FEF6DE770E088E2D3
:1071200090E00E94C20B82E08093D5064EE150E0D1
:1071300060E872E06DC048E8E42E45E0F42E02E01D
:107140002FE130E04FEF5FEF6DE770E088E290E015
:107150000E94C20BA092D5064EE150E062E672E0BA
:1071600057C03EE7E32E35E0F32E02E02FE130E09A
:107170004FEF5FEF6DE770E088E290E00E94C20B96
:10718000B092D50644E150E064E472E041C024E7E7
:10719000E22E25E0F22E02E02FE130E04FEF5FEF2C
:1071A0006DE770E088E290E00E94C20BD093D506B4
:1071B0004EE150E066E272E02BC09AE6E92E95E0DF
:1071C000F92E02E02FE130E04FEF5FEF6DE770E066
:1071D00088E290E00E94C20BC092D5064EE150E0DA
:1071E00068E072E015C080E6E82E85E0F82E02E047
:1071F0002FE130E04FEF5FEF6DE770E088E290E065
:107200000E94C20BD092D5064EE150E06AEE71E0CA
:1072100085E596E00E94E6468FE59AEE0197F1F744
:1072200000C0000080919F0681110FC0A895C093F7
:10723000AB0610928C0610928B06C0939A068FE1D3
:1072400090E00E94420C0E94DC2580919F068130D4
:1072500009F041C0A8958093AB0610928C0610925D
:107260008B0680939A068FE190E00E94420C109268
:10727000E106E091D5068E2F90E08830910540F52B
:10728000FC01E655FF4F4EE150E00C94DB436CEB04
:1072900072E014C06EE972E011C060E872E00EC0E6
:1072A00062E672E00BC064E472E008C066E272E07D
:1072B00005C068E072E002C06AEE71E085E596E024
:1072C0000E94E6468FE59AEE0197F1F700C00000B4
:1072D000A8950E943F2CD0939F06A8959FEF20E78A
:1072E00082E0915020408040E1F700C0000091CE44
:1072F000DF91CF911F910F91FF90EF90DF90CF9092
:10730000BF90AF900895CF93C1E080917306811133
:1073100041C1E091D0068E2F90E08E30910508F0AB
:1073200030C1FC01EE54FF4F0C94DB4360915506D5
:107330007091560670934706609346068EE591E07D
:107340000E9437089093470680934606909356060E
:10735000809355060DC16091570670915806709341
:1073600097066093960682EC91E00E94370890930E
:107370009706809396069093580680935706F8C018
:107380006091590670915A066093DD06772789E16E
:1073900090E00E9437088093DD06992790935A0663
:1073A00080935906E5C060915B0670915C0660931E
:1073B0008206772789E190E00E9437088093820651
:1073C000992790935C0680935B06D2C080915D06FE
:1073D0008093AA060E9446098093AA0690E09093A3
:1073E0005E0680935D06C4C060915F067091600682
:1073F00060938106772788EC90E00E94370880939D
:10740000810699279093600680935F06B1C06091D2
:1074100061067091620660939006772784E690E09B
:107420000E94370880939006992790936206809374
:1074300061069EC0609163067091640660938F063A
:10744000772784E690E00E94370880938F0699277B
:1074500090936406809363068BC060916D06709173
:107460006E067093CC066093CB0688EC90E00E9489
:1074700037089093CC068093CB0690936E0680934A
:107480006D0676C060916F06709170067093540619
:107490006093530684E690E00E9437089093540668
:1074A000809353069093700680936F0661C080911D
:1074B0006506809342060E944609823018F4809344
:1074C000420602C0109242068091420690E09093DC
:1074D0006606809365064CC080914206811103C008
:1074E0001092D0064EC0813009F04BC06091670603
:1074F000709168067093CE066093CD068AEF90E097
:107500000E9437089093CE068093CD06909368062C
:10751000809367062DC080914206882309F381304D
:1075200081F56091690670916A066093A9067727D4
:1075300086E490E00E9437088093A90699279093EB
:107540006A068093690614C0609171067091720694
:10755000709379066093780684E893E00E94370878
:1075600090937906809378069093720680937106C3
:107570002FE788E391E0215080409040E1F700C080
:107580000000C09373061092E1060E945D080E94FD
:107590003F2CBBCECF910895EF92FF920F931F9394
:1075A000CF93DF93A8958091AB068111F5C08FE151
:1075B00090E00E94420C0E943E158091830690E06C
:1075C000909386068093850685E080939F06C1E0B0
:1075D000D5E08091AB068111DFC0A8950E94CF1540
:1075E00080919F068230A9F480918506909186064D
:1075F000019690938606809385060FE110E02CE3B8
:1076000030E046EE50E069E670E081E090E00E94F4
:10761000CD0A80919F068330A9F4809185069091D0
:107620008606019790938606809385060FE110E009
:107630002CE330E046EE50E069E670E081E090E057
:107640000E94CD0A8091850690918606039720F0CE
:107650001092860610928506A895809185069091D5
:1076600086068130910589F1D0F0029709F046C075
:107670008EE7E82E85E0F82E02E02FE130E04FEFB4
:107680005FEF6DE770E088E290E00E94C20B82E05D
:10769000809383064EE150E060E971E02BC022E95F
:1076A000E22E25E0F22E02E02FE130E04FEF5FEF17
:1076B0006DE770E088E290E00E94C20B10928306B2
:1076C0004EE150E06CEC71E015C098E8E92E95E0D1
:1076D000F92E02E02FE130E04FEF5FEF6DE770E051
:1076E00088E290E00E94C20BC09383064EE150E016
:1076F0006EEA71E085E596E00E94E64680919F067D
:1077000081110FC0A895C093AB0610928C06109201
:107710008B06C0939A068FE190E00E94420C0E9473
:10772000DC2580919F06813059F5A8958093AB06A2
:1077300010928C0610928B0680939A068FE190E04F
:107740000E94420C1092E10680918306813069F01C
:1077500038F0823091F44EE150E060E971E009C008
:107760004EE150E06CEC71E004C04EE150E06EEA96
:1077700071E085E596E00E94E646A8950E943F2CC0
:10778000D0939F062FEF80E792E0215080409040F9
:10779000E1F700C000001DCFDF91CF911F910F9145
:1077A000FF90EF900895EF92FF920F931F93CF9366
:1077B000DF93A8958091AB068111F5C08FE190E031
:1077C0000E94420C0E943E1580918A0690E09093A0
:1077D00086068093850685E080939F06C1E0D5E00C
:1077E0008091AB068111DFC0A8950E94CF158091D2
:1077F0009F068230A9F480918506909186060196B5
:1078000090938606809385060FE110E02CE330E02C
:1078100046EE50E069E670E081E090E00E94CD0A1B
:1078200080919F068330A9F4809185069091860609
:10783000019790938606809385060FE110E02CE374
:1078400030E046EE50E069E670E081E090E00E94B2
:10785000CD0A8091850690918606039720F01092BC
:107860008606109285068091850690918606813065
:10787000910589F1D0F0029709F046C08EE7E82E15
:1078800085E0F82E02E02FE130E04FEF5FEF6DE78B
:1078900070E088E290E00E94C20B82E080938A064A
:1078A0004EE150E066E371E02BC022E9E22E25E0D4
:1078B000F22E02E02FE130E04FEF5FEF6DE770E076
:1078C00088E290E00E94C20B10928A064EE150E0DE
:1078D00062E771E015C098E8E92E95E0F92E02E024
:1078E0002FE130E04FEF5FEF6DE770E088E290E06E
:1078F0000E94C20BC0938A064EE150E064E571E03D
:1079000085E596E00E94E64680919F06811110C0B1
:10791000A895C093AB0610928C0610928B06C0936C
:107920009A068FE190E00E94420CA8950E94DC2507
:1079300080919F06813059F5A8958093AB061092EF
:107940008C0610928B0680939A068FE190E00E943D
:10795000420C1092E10680918A06813069F038F07D
:10796000823091F44EE150E066E371E009C04EE1EF
:1079700050E062E771E004C04EE150E064E571E080
:1079800085E596E00E94E646A8950E943F2CD0939C
:107990009F062FEF80E792E0215080409040E1F772
:1079A00000C000001DCFDF91CF911F910F91FF907C
:1079B000EF900895EF92FF920F931F93CF93DF9371
:1079C000A8958091AB068111F6C08FE190E00E94EE
:1079D000420C0E943E158091DF0690E0909386064F
:1079E0008093850685E080939F06C1E0D5E0809175
:1079F000AB068111E0C0A8950E94CF1580919F062B
:107A00008230A9F480918506909186060196909324
:107A10008606809385060FE110E02CE330E046EE09
:107A200050E069E670E081E090E00E94CD0A80912C
:107A30009F068330A9F48091850690918606019770
:107A400090938606809385060FE110E02CE330E0EA
:107A500046EE50E069E670E081E090E00E94CD0AD9
:107A60008091850690918606039720F010928606F5
:107A70001092850680918506909186068130910549
:107A800089F1D0F0029709F046C08EE7E82E85E034
:107A9000F82E02E02FE130E04FEF5FEF6DE770E08E
:107AA00088E290E00E94C20B82E08093DF064EE104
:107AB00050E06CED70E02BC022E9E22E25E0F22EC2
:107AC00002E02FE130E04FEF5FEF6DE770E088E21A
:107AD00090E00E94C20B1092DF064EE150E068E198
:107AE00071E015C098E8E92E95E0F92E02E02FE14B
:107AF00030E04FEF5FEF6DE770E088E290E00E94CA
:107B0000C20BC093DF064EE150E06AEF70E085E5FE
:107B100096E00E94E64680919F06811110C0A895CC
:107B2000C093AB0610928C0610928B06C0939A06F7
:107B30008FE190E00E94420CA8950E94DC25809184
:107B40009F06813061F5A8958093AB0610928C0654
:107B500010928B0680939A068FE190E00E94420C6F
:107B6000A8951092E1068091DF06813069F038F027
:107B7000823091F44EE150E06CED70E009C04EE1CE
:107B800050E068E171E004C04EE150E06AEF70E05F
:107B900085E596E00E94E646A8950E943F2CD0938A
:107BA0009F062FEF80E792E0215080409040E1F760
:107BB00000C000001CCFDF91CF911F910F91FF906B
:107BC000EF9008950F931F9380917C06811199C0C7
:107BD0008091D7069091D8068335910591F581E083
:107BE00080937C060E943A1B0FE110E02CE330E00A
:107BF00044E650E06BE470E08EE690E00E94CD0A2F
:107C000024E230E04AE550E064E670E088E090E08D
:107C10000E94CD0A24E230E04AE550E064E670E0DC
:107C200088E090E00E94CD0A24E230E04AE550E08E
:107C300064E670E08FED90E00E94CD0A0E94DC25A2
:107C4000A8950E94B8240E948D20A89503E02FE1FA
:107C500030E04FEF5FEF69E170E085E890E00E946F
:107C60007D190E9466240E944A1180917C06813011
:107C7000A9F5A8950E943A1B0FE110E02CE330E033
:107C800044E650E06BE470E08EE690E00E94CD0A9E
:107C900024E230E04AE550E064E670E088E090E0FD
:107CA0000E94CD0A24E230E04AE550E064E670E04C
:107CB00088E090E00E94CD0A24E230E04AE550E0FE
:107CC00064E670E08FED90E00E94CD0A809141065D
:107CD000813009F4CCD10E94DC25A8952FEF81EEEC
:107CE00094E0215080409040E1F700C000000E94E5
:107CF000D3170E948F240E9455181F910F910C9446
:107D0000C5181F910F9108951F920F920FB60F92F1
:107D100011248F939F938CB190E09093D806809319
:107D2000D7069F918F910F900FBE0F901F901895BF
:107D30001F920F920FB60F9211242F938F939F9340
:107D400080914F06909150060196883E23E092075D
:107D500028F49093500680934F0604C0109250066A
:107D600010924F0680917A06811105C01092DA06B2
:107D70001092D9060BC0813049F48091D9069091B8
:107D8000DA0601969093DA068093D90680919406DC
:107D9000811105C010924E0610924D060BC0813025
:107DA00049F480914D0690914E06019690934E06AF
:107DB00080934D0680918D06811105C01092520668
:107DC000109251060BC0813049F480915106909178
:107DD0005206019690935206809351069F918F917F
:107DE0002F910F900FBE0F901F9018952FEF89E6DF
:107DF00098E1215080409040E1F700C000008FEFF3
:107E00008ABB81BB80936100C1E0C4BB88EA8FBD9F
:107E10008CE08EBD1DBC1CBC17BC16BC8AE78BBD9C
:107E200082E18ABD19BC18BC1092790010927800CA
:107E300080E187BF10BE87E683BF12BE11BE81E816
:107E400080938B0085E080938A00109289001092C5
:107E5000880010928100109280001092870010928A
:107E60008600109285001092840010928300109278
:107E700082001BB888E98AB986E080939500109249
:107E800090008FE289B98FE181BD8FE081BDE3D29F
:107E900081E00E94D9098FE190E00E94420CC093DA
:107EA0007C0610927D061092500610924F0610929A
:107EB000920610924C0610927B061092DB061092EE
:107EC000740680E590E09093D8068093D706809161
:107ED00064008E7F80936400809165008160809350
:107EE00065008091640088608093640080916500E3
:107EF000886080936500C093410680916400826031
:107F0000809364008091650082608093650078941E
:107F1000A49AAC9A2FEF85EA9EE0215080409040D1
:107F2000E1F700C00000A895AC988AED92E05ED71A
:107F3000813079F00E94D820A8950E944524A89508
:107F400061E08BED92E068D7A89561E08AED92E060
:107F500063D7A89580917C06813021F4A8950E9472
:107F6000DC25A895A8952EDEF4CF80916400806171
:107F700080936400809165008061809365008091AA
:107F8000640088608093640080916500877F80939F
:107F900065008091390690913A068536910500F585
:107FA00080916400846080936400809165008460A7
:107FB000809365008FEC97E00197F1F700C0000017
:107FC000A895809165008B7F80936500809139062C
:107FD00090913A06019690933A0680933906D9CF4C
:107FE00080916500886080936500089580916400A9
:107FF000806180936400809165008F7E809365002E
:108000008091640088608093640080916500877F20
:10801000809365008091390690913A0685369105E6
:1080200000F5809164008460809364008091650015
:108030008460809365008FEC97E00197F1F700C0B2
:108040000000A895809165008B7F809365008091EA
:10805000390690913A06019690933A068093390634
:10806000D9CF80916500886080936500089582EE85
:1080700092E0BCD68093E306809164008061809397
:108080006400809165008061809365008091640048
:1080900088608093640080916500877F809365008D
:1080A0008091E30624E6829FC001112420913706C7
:1080B000309138062817390700F5809164008460F4
:1080C00080936400809165008460809365008FECEC
:1080D00097E00197F1F700C00000A8958091650036
:1080E0008B7F8093650080913706909138060196CA
:1080F0009093380680933706D3CF809165008860CF
:108100008093650010923D06109238061092370653
:108110000895AC0180913D0681114AC090916400A0
:10812000906190936400909165009F7E90936500AC
:108130009091640098609093640090916500977F9F
:108140009093650084E6849F9001859F300D1124F3
:1081500080913706909138068217930700F5809139
:1081600064008460809364008091650084608093E3
:1081700065008FEC97E00197F1F700C00000A8952B
:10818000809165008B7F8093650080913706909188
:10819000380601969093380680933706D9CF8091A0
:1081A000650088608093650010923806109237064B
:1081B00081E080933D060895682F82EE92E02CC600
:1081C00082EE92E013D690E0A4CF80933C0608950F
:1081D000CF93DF9300D000D0CDB7DEB7809163009E
:1081E0001C821B821A821982BE016F5F7F4FCE01F3
:1081F000039644D18B819C818431954068F48981B8
:108200009A81843A964040F489819A818D329140D6
:1082100018F082E08093E5068B819C818937954038
:1082200090F08B819C81843C994068F489819A818B
:10823000843A964040F489819A818D32914018F0B9
:1082400083E08093E5068B819C8189329A4068F0B7
:1082500089819A8184379E4040F489819A81813D49
:10826000974018F081E08093E5068B819C81863FE2
:10827000994060F48B819C818134964038F08981EB
:108280009A81813D974010F01092E5068091E506B5
:108290000F900F900F900F90DF91CF910895DF9284
:1082A000EF92FF920F931F93CF93DF9385E080931C
:1082B000E506DBE485E0D82E80913C0681116FC095
:1082C00087DFE0903B06F12C03E02FE130E040E057
:1082D00058EF62E870E080E590E00E94080C809121
:1082E000E5068330B1F480913B06815080933B06D4
:1082F00010923A06109239060FE110E02CE330E0BC
:1083000046EE50E069E670E081E090E00E94CD0A20
:108310002CDE8091E5068230C1F480913B068B34DF
:10832000A0F48F5F80933B0610923A0610923906B4
:108330000FE110E02CE330E046EE50E069E670E03B
:1083400081E090E00E94CD0A51DE80913B068C34A2
:1083500010F0D0933B068091E50681110EC00FE12D
:1083600010E02CE330E046EE50E069E670E081E09A
:1083700090E00E94CD0A10923B06C091E506C13004
:1083800059F480913B0618DF80913B0690E06FDE48
:1083900010923B06C0933C06D092E5068DCFDF914C
:1083A000CF911F910F91FF90EF90DF900895EF9282
:1083B000FF920F931F9382EE92E018D58C3418F43D
:1083C0008093E40612C01092E40660E082EE92E030
:1083D00023D50FE110E028E230E048E550E06FEAF5
:1083E00070E080EE90E00E94CD0A8091E406882340
:1083F00081F082EE92E0FAD4E82EF12C02E02FE137
:1084000030E04FEF5FEF6AEA70E080EF90E00E94AB
:10841000080C1F910F91FF90EF900895EF92FF923B
:108420000F93E090E406F12C02E02FE130E04FEFF3
:108430005FEF6AEA70E080EF90E00E94080C0F9115
:10844000FF90EF900895C098AB9AAF9A8FB9779B41
:10845000FECF8FB1089587E087BBC09AAB9AAF9AE1
:1084600083E58DB91EB880E8EEDF80E0ECDF80E0C8
:10847000EADF8AE18A95F1F700C00895EF92FF9252
:108480000F931F93CF93DF9300D000D0CDB7DEB70B
:108490007C018B01A895AB9AAF9A1C821B821A8231
:1084A000198280EDD0DF80E0CEDF8FB190E09C8339
:1084B0008B838B819C81982F88279C838B8380E082
:1084C000C2DF2FB18B819C81822B9C838B838B811C
:1084D0009C8133E0969587953A95E1F79C838B8351
:1084E00087EC90E00197F1F700C0000080E9ABDF76
:1084F00080E0A9DF8FB190E09A83898389819A8196
:10850000982F88279A83898380E09DDF2FB1898106
:108510009A81822B9A83898389819A8153E09695E7
:1085200087955A95E1F79A8389838B819C81F7011E
:108530009183808389819A81F801918380830F9050
:108540000F900F900F90DF91CF911F910F91FF909F
:10855000EF90089570D088F09F5790F0B92F992729
:10856000B751A0F0D1F0660F771F881F991F1AF03E
:10857000BA95C9F712C0B13081F077D0B1E0089553
:1085800074C0672F782F8827B85F39F0B93FCCF3D4
:10859000869577956795B395D9F73EF49095809534
:1085A000709561957F4F8F4F9F4F0895E89409C054
:1085B00097FB3EF490958095709561957F4F8F4F16
:1085C0009F4F9923A9F0F92F96E9BB279395F6952C
:1085D000879577956795B795F111F8CFFAF4BB0FAA
:1085E00011F460FF1BC06F5F7F4F8F4F9F4F16C00E
:1085F000882311F096E911C0772321F09EE8872F98
:10860000762F05C0662371F096E8862F70E060E053
:108610002AF09A95660F771F881FDAF7880F9695CC
:10862000879597F9089557FD9058440F551F59F0B5
:108630005F3F71F04795880F97FB991F61F09F3F4F
:1086400079F087950895121613061406551FF2CF78
:108650004695F1DF08C0161617061806991FF1CFC8
:1086600086957105610508940895E894BB276627EF
:108670007727CB0197F908950BD078C069D028F0FF
:108680006ED018F0952309F05AC05FC01124EECFC8
:10869000CADFA0F3959FD1F3950F50E0551F629F5D
:1086A000F001729FBB27F00DB11D639FAA27F00D4B
:1086B000B11DAA1F649F6627B00DA11D661F829F72
:1086C0002227B00DA11D621F739FB00DA11D621F57
:1086D000839FA00D611D221F749F3327A00D611D74
:1086E000231F849F600D211D822F762F6A2F112456
:1086F0009F5750408AF0E1F088234AF0EE0FFF1FA9
:10870000BB1F661F771F881F91505040A9F79E3FDF
:10871000510570F014C0AACF5F3FECF3983EDCF334
:10872000869577956795B795F795E7959F5FC1F71C
:10873000FE2B880F911D9695879597F9089597F9C7
:108740009F6780E870E060E008959FEF80EC0895F7
:1087500000240A9416161706180609060895002420
:108760000A9412161306140605060895092E03949A
:10877000000C11F4882352F0BB0F40F4BF2B11F40E
:1087800060FF04C06F5F7F4F8F4F9F4F0895AA1BFC
:10879000BB1B51E107C0AA1FBB1FA617B70710F0EC
:1087A000A61BB70B881F991F5A95A9F7809590951E
:1087B000BC01CD010895EE0FFF1F0024001C0BBE6D
:1087C0000790F691E02D0994A29FB001B39FC001DC
:1087D000A39F700D811D1124911DB29F700D811DED
:1087E0001124911D0895BB274A3031F4992322F4B6
:1087F000BDE2909581959F4F01C0BB27FB01552796
:10880000AA27880F991FAA1FA41710F0A41B8395ED
:108810005051B9F7A05DAA3308F0A95DA193009764
:1088200079F7B111B1931192CB0126C2CF93DF93A7
:10883000CDB7DEB7AE014B5F5F4FFA016191719129
:10884000AF018091E8069091E90603D0DF91CF91C6
:1088500008952F923F924F925F926F927F928F92E4
:108860009F92AF92BF92CF92DF92EF92FF920F93BF
:108870001F93CF93DF93CDB7DEB72B970FB6F89446
:10888000DEBF0FBECDBF6C017B018A01FC011782E8
:108890001682838181FFBFC1CE0101963C01F601A2
:1088A0009381F70193FD859193FF81917F01882347
:1088B00009F4ADC1853239F493FD859193FF81911F
:1088C0007F01853221F4B60190E0E6D1E8CF912C0A
:1088D000212C312CFFE1F315D8F08B3279F038F4EC
:1088E000803279F08332A1F4232D20611DC08D32B6
:1088F00061F0803369F4232D216016C0832D8260DE
:10890000382EE32DE4603E2E2AC0F32DF8601DC002
:1089100037FC2DC020ED280F2A3040F08E32B9F4FC
:1089200036FC75C1232D2064322E19C036FE06C0D8
:108930008AE0989E200D1124922E11C0EAE02E9E0E
:10894000200D1124222EF32DF0623F2E08C08C360C
:1089500021F4832D8068382E02C0883641F4F70157
:1089600093FD859193FF81917F018111B3CF982F62
:108970009F7D9554933028F40C5F1F4F9FE399839C
:108980000DC0833631F0833771F0833509F055C05F
:1089900020C0F801808189830E5F1F4F8824839453
:1089A000912C530112C02801F2E04F0E511CF80126
:1089B000A080B18036FE03C0692D70E002C06FEF69
:1089C0007FEFC5014ED14C018201F32DFF773F2E81
:1089D00015C0280122E0420E511CF801A080B18090
:1089E00036FE03C0692D70E002C06FEF7FEFC50156
:1089F0002DD14C01F32DF0683F2E820133FC19C0BC
:108A0000822D90E088169906A0F4B60180E290E0ED
:108A100043D12A94F5CFF50137FC859137FE81913A
:108A20005F01B60190E038D121102A9421E0821A2A
:108A300091088114910479F7E1C0843611F08936E8
:108A400039F5F80137FE07C0608171818281938119
:108A50000C5F1F4F08C060817181072E000C880BCE
:108A6000990B0E5F1F4FF32DFF763F2E97FF09C026
:108A700090958095709561957F4F8F4F9F4FF068CF
:108A80003F2E2AE030E0A30143D1882E861844C04F
:108A9000853731F4232D2F7EB22E2AE030E025C019
:108AA000932D997FB92E8F36C1F018F4883579F05F
:108AB000AEC0803719F0883721F0A9C0E92FE061F6
:108AC000BE2EB4FE0DC0FB2DF460BF2E09C034FED7
:108AD0000AC0292F2660B22E06C028E030E005C06B
:108AE00020E130E002C020E132E0F801B7FE07C02B
:108AF00060817181828193810C5F1F4F06C060810C
:108B0000718180E090E00E5F1F4FA30101D1882E9C
:108B10008618FB2DFF773F2E36FE0DC0232D2E7FAE
:108B2000A22E891458F434FE0BC032FC09C0832DE8
:108B30008E7EA82E05C0B82CA32C03C0B82C01C073
:108B4000B92CA4FE0FC0FE01E80DF11D8081803319
:108B500021F49A2D997EA92E09C0A2FE06C0B394D5
:108B6000B39404C08A2D867809F0B394A3FC10C096
:108B7000A0FE06C0B21480F4280C922C9B180DC0E5
:108B8000B21458F4B60180E290E086D0B394F8CFE6
:108B9000B21418F42B1802C0982C212CA4FE0FC07C
:108BA000B60180E390E078D0A2FE16C0A1FC03C01D
:108BB00088E790E002C088E590E0B6010CC08A2DFD
:108BC000867851F0A1FE02C08BE201C080E2A7FCD2
:108BD0008DE2B60190E060D0891430F4B60180E3F4
:108BE00090E05AD09A94F8CF8A94F301E80DF11DE1
:108BF0008081B60190E050D08110F6CF222009F498
:108C00004ECEB60180E290E047D02A94F7CFF6012D
:108C10008681978102C08FEF9FEF2B960FB6F89455
:108C2000DEBF0FBECDBFDF91CF911F910F91FF909F
:108C3000EF90DF90CF90BF90AF909F908F907F90FC
:108C40006F905F904F903F902F900895FC0105909A
:108C5000615070400110D8F7809590958E0F9F1F3E
:108C60000895FC016150704001900110D8F7809583
:108C700090958E0F9F1F0895DC01FC01672F719165
:108C80007723E1F7329704C07C916D9370836291F2
:108C9000AE17BF07C8F308950F931F93CF93DF93C9
:108CA000FB01238121FD03C08FEF9FEF2CC022FF2A
:108CB00016C046815781248135814217530744F4F9
:108CC000A081B1819D012F5F3F4F318320838C9321
:108CD000268137812F5F3F4F3783268314C08B0156
:108CE000EC01FB010084F185E02D0995892BE1F66B
:108CF000D80116968D919C911797019617969C9383
:108D00008E931697CE01DF91CF911F910F91089509
:108D1000FA01AA27283051F1203181F1E8946F93AC
:108D20006E7F6E5F7F4F8F4F9F4FAF4FB1E03ED052
:108D3000B4E03CD0670F781F891F9A1FA11D680FF0
:108D4000791F8A1F911DA11D6A0F711D811D911D23
:108D5000A11D20D009F468943F912AE0269F112498
:108D60003019305D3193DEF6CF010895462F4770FC
:108D7000405D4193B3E00FD0C9F7F6CF462F4F7057
:108D8000405D4A3318F0495D31FD4052419302D0B5
:108D9000A9F7EACFB4E0A69597958795779567955B
:108DA000BA95C9F700976105710508959B01AC015B
:108DB0000A2E06945795479537952795BA95C9F782
:108DC000620F731F841F951FA01D0895DC01CB0146
:108DD000FC01E199FECF06C0FFBBEEBBE09A3196E5
:108DE0000DB20D9241505040B8F70895E199FECF71
:108DF0009FBB8EBBE09A99278DB30895A8E1B0E0A0
:108E000042E050E0E5CFDC01CB0102C02D9105D05E
:108E100041505040D8F70895262FE199FECF9FBBCF
:108E20008EBB2DBB0FB6F894E29AE19A0FBE019665
:0C8E30000895F2DF272FF1CFF894FFCF58
:108E3C00140048005D0078009600B600D500F300E1
:108E4C0010012C01490163017C019401AC01C101A9
:108E5C00D501E801010E00000002000000002A0FFD
:108E6C000000000044656C004F4E004F4646002049
:108E7C0020D1F2E0EDF6E8FF00C2E5F0F5EDE8E90F
:108E8C0000CDE8E6EDE8E900D0F3F7EDEEE900D02F
:108E9C00E5E1EEEBEBE8EDE32000D1F3F8EAE000DE
:108EAC00ECE8EAF0EEF1F5E5EC00EFEBE0F200CAED
:108EBC00E0EBE8E1F0EEE2EAE000EDE8E7E000CC20
:108ECC00EEF9EDEEF1F2FC00E2E5F0F5E000C2E5C2
:108EDC00F0F5EDE8E920EDE0E3F02E00CDE8E6ED6D
:108EEC00E8E920EDE0E3F02E20002020D0F3F7EDB0
:108EFC00EEE92020200020D1F3F8EAE020EFEBE0AF
:108F0C00F22000C4EEEF2E20EDE0F1F2F0EEE9EAF3
:108F1C00E8002020D1F2E5EAEBEE00CAE0EBE8E154
:108F2C00F0EEE2EAE02000EDE8E7E02000C2DBD55D
:108F3C00CEC40057543D2025750A47530047533D76
:108F4C002025750A534E00534E3D2025750A454E7B
:108F5C004400574B3D2025750A565000503D332E8A
:108F6C00360A5200524C3D2025750A68004F3D735D
:108F7C00740A5300473D73740A530053523D5374A3
:108F8C006174696F6E200A57500057503D536E360E
:108F9C00332F506233370A57540057503D536E41AC
:108FAC00670A57540057503D50726F66696C6530B4
:108FBC000A57540057503D50726F66696C65310A00
:108FCC0057540057503D50726F66696C65320A57A2
:108FDC00540057503D50726F66696C65330A575494
:108FEC000057503D50726F66696C65340A575400D7
:108FFC0057503D50726F66696C65350A5754005373
:10900C00523D5550686561746572200A5750005383
:10901C00523D507265686561746572200A57500044
:10902C0053523D4D616E75616C200A57500053527E
:10903C003D5265626F6C6C696E67200A5750005325
:10904C00523D4368697068656174696E67200A57A0
:10905C00500053523D50434268656174696E6720FD
:10906C000A57500053523D5043200A575000C2FB40
:10907C00E1E5F0E8F2E520E2FBF1EEF2F300563523
:10908C002E307A00202020C2F0E5ECFF20F0E5E144
:10909C00EEEBEBE8EDE3E02020202000C2FBE1E565
:1090AC00F0E8F2E520F0E5E6E8EC00D2E5ECEFE5DF
:1090BC00F0E0F2F3F0E020EFEEEBEEF7EAE8202040
:1090CC0000EDE8E7E020EFF0E820E4EEEDE0E3F07F
:1090DC00E5E2E500D2E5ECEFE5F0E0F2F3F0E020BC
:1090EC00F3E2E5EBE8F7E5EDE8FF00202020202097
:1090FC0020E4EEEDE0E3F0E5E2E02020202020206B
:10910C0000C4EBE8F2E5EBFCEDEEF1F2FC20E2EF53
:10911C00E8F2FBE2E0EDE8FF00D4F3EDEAF6E8FF5D
:10912C0020E4EEEDEEE3F0E5E2E000EDE8E6EDE55F
:10913C00E3EE20EDE0E3F0E5E2E0F2E5EBFF2020EA
:10914C00202000CCE0EAF1E8ECE0EBFCEDE0FF20C5
:10915C00ECEEF9EDEEF1F2FC202000E2E5F0F5ED9D
:10916C00E5E3EE20EDE0E3F0E5E2E0F2E5EBFF20F5
:10917C00202000CCE0EAF1E8ECE0EBFCEDE0FF2095
:10918C00ECEEF9EDEEF1F2FC202000E2E5F0F5ED6D
:10919C00E5E3EE20EDE0E3F0E5E2E0F2E5EBFF20C5
:1091AC00202000D2E5ECEFE5F0E0F2F3F0E020E275
:1091BC00EAEBFEF7E5EDE8FF202000CAEEEDF2F059
:1091CC00EEEBFC20EFEE20E2E5F0F5F32020202082
:1091DC00202000EDE8E6EDE5E3EE20EDE0E3F0E540
:1091EC00E2E0F2E5EBFF2020202000CAEEFDF4F4D3
:1091FC00E8F6E8E5EDF220EFF0EEF4E8EBFF2020E6
:10920C00202000E2E5F0F5EDE5E3EE20EDE0E3F003
:10921C00E5E2E0F2E5EBFF20202000CAEEFDF4F4DD
:10922C00E8F6E8E5EDF220EFF0EEF4E8EBFF2020B5
:10923C00202000EDE0E3F0E5E2E0F2E5EBFF20209A
:10924C0000D2E5ECEFE5F0E0F2F3F0E020EDE8E63B
:10925C00EDE5E3EE2020202000EFE0E9EAE8200035
:10926C00D2E5ECEFE5F0E0F2F3F0E020ECE5F1F222
:10927C00E0202020202000C2FBE1E5F0E8F2E52010
:10928C00EFF0EEF4E8EBFC0036302D393020D10055
:10929C00CFF0EEF4E8EBFC203500CFF0EEF4E8EB89
:1092AC00FC203400CFF0EEF4E8EBFC203300CFF0E0
:1092BC00EEF4E8EBFC203200CFF0EEF4E8EBFC200F
:1092CC003100CFF0EEF4E8EBFC203000536E416738
:1092DC0000536E506200CFF0E8EDFFF2EE2020005C
:1092EC00C2DBC1D0C0D2DC00C2DBCACB00C2CACB4D
:1092FC0000CDE0F1F2F0EEE8F2FC00C7E2F3EAEEAA
:10930C00E2FBE520F1E8E3EDE0EBFB00CFF0E5E478
:10931C00F3F1F2E0EDEEE2EAE800D3ECEEEBF7E08D
:10932C00EDE8FF00C2F0E5ECFF20EFE0E9EAE80031
:10933C0020C4E0F2F7E8EA20EDE8E62E20EDE0E3C9
:10934C00F0E5E2E0F2E5EBFF0020C4E0F2F7E8EA3A
:0E935C0020ECE5F1F2E020EFE0E9EAE80000A5
:00000001FF
